:020000040001F9
:10C0000040460020C1C30100C9C30100CBC30100E9
:10C01000CDC30100CFC30100D1C301000000000067
:10C02000000000000000000000000000D3C3010079
:10C03000D5C3010000000000D7C30100D9C301002F
:10C0400031C60100DBC30100D5C80100DBC301001C
:10C05000DBC30100DBC301008DC50100DBC30100B0
:10C06000DBC30100DBC30100DBC30100DBC3010054
:10C07000DBC30100DBC30100DBC30100DBC3010044
:10C08000DBC3010081C60100DBC30100DBC301008B
:10C09000DBC30100DBC30100F1C60100DBC301000B
:10C0A000DBC30100DBC30100DBC30100DBC3010014
:10C0B000DBC30100DBC30100000000000000000042
:10C0C000DBC30100DBC30100DBC30100DBC30100F4
:10C0D000DBC30100DBC30100DBC30100DBC30100E4
:10C0E000DBC30100000000000000000000000000B1
:10C0F00000000000DBC3010000000000DBC3010002
:10C10000000000000000000000000000000000002F
:10C11000000000000000000000000000000000001F
:10C12000000000000000000000000000000000000F
:10C1300000000000000000000000000000000000FF
:10C1400000000000000000000000000000000000EF
:10C1500000000000000000000000000000000000DF
:10C1600000000000000000000000000000000000CF
:10C1700000000000000000000000000000000000BF
:10C1800000000000000000000000000000000000AF
:10C19000000000000000000000000000000000009F
:10C1A000000000000000000000000000000000008F
:10C1B000000000000000000000000000000000007F
:10C1C000000000000000000000000000000000006F
:10C1D000000000000000000000000000000000005F
:10C1E000000000000000000000000000000000004F
:10C1F000000000000000000000000000000000003F
:10C20000DFF80CD000F084F9004800479DE90100F8
:10C210004046002030B450E8012F93B2C489234433
:10C220008489A34228BF1B1B0489A34202BFBFF31A
:10C230002F8F002007E0C3EA020340E80134002CFE
:10C24000E9D14FF001000A6030BC704750E8012F7F
:10C25000C2EA024240E801210029F7D1704730B418
:10C2600050E8022F1FFAA2F3C488A34202BFBFF313
:10C270002F8F00200DE0C48923448489A34228BF66
:10C280001B1BC2EA034340E80234002CE8D14FF004
:10C2900001000A6030BC704750E8022FC2EA224217
:10C2A00040E802210029F7D17047034653E8022FE6
:10C2B000D988B2EB324F4FF0000017BF92B241EA7B
:10C2C000014142EA014104E05A68B2EB324F08BF33
:10C2D000012043E80212002AE8D1704730B4044636
:10C2E00054E8000F0D4644E80053002BF8D11560C8
:10C2F00030BC704730B4044654E8000F40EA0105F2
:10C3000044E80053002BF7D1156030BC704730B4BF
:10C31000044654E8000F00EA010544E80053002BEE
:10C32000F7D1156030BC704730B4044654E8000FB4
:10C3300080EA010544E80053002BF7D1156030BCBA
:10C34000704730B4044654E8000F00EB010544E8A0
:10C350000053002BF7D1156030BC704730B4044651
:10C3600054E8000FA0EB010544E80053002BF7D17F
:10C37000156030BC704770B404464FF0000054E8BC
:10C38000006F0D68AE4207BF44E80023012044E877
:10C3900000630E60002B1CBF0020F0E770BC7047EC
:10C3A00030B4044654E8000F88422CBF451A0546B5
:10C3B00044E80053002BF5D1156030BC70470000F5
:10C3C0000648804706480047FEE7FEE7FEE7FEE72F
:10C3D000FEE7FEE7FEE7FEE7FEE7FEE7F5C6010043
:10C3E00001C201002DE9F05F0546002092469B4600
:10C3F00088460646814640241BE02846414647467B
:10C40000224600F074F853465A46C01A914110D3A0
:10C4100011461846224600F016F82D1A67EB01085F
:10C420004F4622460120002100F00DF817EB0009CD
:10C430004E41201EA4F10104DFDC484631462A4665
:10C440004346BDE8F09F202A04DB203A00FA02F1BF
:10C45000002070479140C2F1200320FA03F31943F2
:10C4600090407047004870471C29020040EA0103D1
:10C470009B0703D009E008C9121F08C0042AFAD29A
:10C4800003E011F8013B00F8013B521EF9D270475E
:10C49000D2B201E000F8012B491EFBD27047002206
:10C4A000F6E710B513460A4604461946FFF7F0FFB3
:10C4B000204610BD421C10F8011B0029FBD1801A38
:10C4C000704730B504460020034600E05B1C9342F1
:10C4D00003D2E05CCD5C401BF8D030BD034611F8C0
:10C4E000012B00F8012B002AF9D118467047202AA9
:10C4F00004DB203A21FA02F00021704721FA02F30E
:10C50000D040C2F120029140084319467047000014
:10C51000064C074D06E0E06840F0010394E8070090
:10C5200098471034AC42F6D3FFF76EFE4C31020050
:10C530006C31020070B58C1810F8015B15F0070320
:10C5400001D110F8013B2A1106D110F8012B03E0AC
:10C5500010F8016B01F8016B5B1EF9D12B0705D4B4
:10C560000023521E0DD401F8013BFAE710F8013BFD
:10C57000CB1A921C03E013F8015B01F8015B521E19
:10C58000F9D5A142D8D3002070BD00002DE9FC41AF
:10C590000025DFF8948000954FF4807601242F4623
:10C5A0000195304603F0BAF938B1D8F804032042B7
:10C5B00003D0304603F0A8F92543361D64007F1CE4
:10C5C000B6B2082FEDD34FF4BE74204603F0A6F99F
:10C5D00048B1204603F098F945F000456A4602212B
:10C5E000002003F0F9F815F0FF0F16D00126002403
:10C5F0002E420ED008EB8401D1F81005D1F81015A9
:10C60000C0F30520094AC1F3014152F8242002B1C8
:10C6100090477600641C082CEAD3002D02DA6846A5
:10C6200004F0E4FEBDE8FC810060004064340020BA
:10C6300070B54FF48076304602F088FE0F4DB40599
:10C6400040B1304602F089FE0120C4F80803296891
:10C65000002088474FF48276304602F077FE0028AB
:10C660000AD0304602F079FE0220C4F80803296897
:10C67000BDE870400120084770BD0000EC2D00208F
:10C6800002490248091F0968006808475C2E00201B
:10C6900000F026B970B50E46144900EB400001EBDE
:10C6A000C0051446E86A183520B101280FD00228C9
:10C6B00005D113E0284600F047F9A04201D200243A
:10C6C00011E022463146284600F076F90BE0284674
:10C6D00000F03AF9A042F4D20446F2E73146284687
:10C6E00000F03DF90446204670BD0000B83B002034
:10C6F00003F056BFF0B54FF080516A4ED1F83001CB
:10C70000694D421C07D0D1F834310746012400227C
:10C710000D2F05D00FE02A783778C2F30313F5E721
:10C720000BB1012B07D14FF08043C3F80C21C3F8A4
:10C7300010215E4B1A60431C05D0D1F834710346BA
:10C740000D2B05D05DE02F783378C7F30317F7E79B
:10C750000FB1012F55D1564B1B68564F3B60544BC0
:10C760001B1D1B683F1D3B60514B08331B683F1D61
:10C770003B604F4B0C331B683F1D3B604C4B1033F1
:10C780001B683F1D3B604A4B14331B683F1D3B60D9
:10C79000474B18331B68474F20373B60444B1C33D3
:10C7A0001B683F1D3B60424B20331B683F1D3B60B5
:10C7B0003F4B24331B683F1D3B603D4B28331B68B8
:10C7C0003F1D3B603A4B2C331B683F1D3B60384B91
:10C7D00030331B68374F40373B60354B34331B6871
:10C7E0003F1D3B60324B38331B683F1D3B60304B75
:10C7F0003C331B683F1D3B602D4B40331B683F1D86
:10C800003B60431C04D0D1F834110D2805D00EE054
:10C8100029783078C1F30311F7E709B1012906D16E
:10C8200025480168C90702D06FF001010160234863
:10C83000016841F470010160BFF34F8FBFF36F8F48
:10C840004FF01020D0F80012002903DBD0F80412BA
:10C85000002922DA1A4B1C601A490C68002CFCD003
:10C860001224C0F800420D68002DFCD0C0F804422C
:10C8700008680028FCD01A6008680028FCD0BFF3C4
:10C880004F8F0E487C3801680F4A01F4E061114374
:10C890000160BFF34F8F00BFFDE70D490B480860F3
:10C8A000F0BD0000E00F00F0E80F00F03805004098
:10C8B0000404001020C500400004004088ED00E0A2
:10C8C00004E5014000E401400400FA050090D003B3
:10C8D000D42E00200148006800470000F42D0020FD
:10C8E00010B5124C02202061606111A0A06104F11A
:10C8F0007800E0614FF4007020620020A062606266
:10C900000BA1A164E06204F51E71E1641021A06531
:10C91000C4E91410E06509A1E01DFFF7DFFD08A1DF
:10C920002046FFF7DBFD2020A07110BDB83B0020A2
:10C930005465726D696E616C0000000052545400C1
:10C9400053454747455200000269C1688A4203D8EF
:10C950008068401A104400E0501A401E70472DE9CC
:10C96000F047C4681746894606464FF0000830690C
:10C97000A04201D9051B02E0B168201A0D1AB06867
:10C980006D1E001BA84200D80546BD4200D33D469F
:10C9900070682A4620444946FFF768FDB0687F1B4F
:10C9A0002C44A844A944A04200D10024F460002FE4
:10C9B000DDD14046BDE8F0872DE9F04104468846C8
:10C9C000D4E90207C51BE168606816460844B54211
:10C9D00006D94146FFF74AFDB819E060BDE8F0818D
:10C9E0002A464146FFF742FD761B08EB0501324619
:10C9F0006068FFF73BFDE660F0E70000014A02498E
:10CA000000F026B827E501006C2E002002E008C8DF
:10CA1000121F08C1002AFAD170477047002001E0B8
:10CA200001C1121F002AFBD17047000001212028FC
:10CA300003DA81400548014003E0402802DA20384B
:10CA4000814009B10120704700207047FC06FFBDFE
:10CA50002DE9F04116460F460446002503E039460D
:10CA6000B047641C6D1C20780028F8D12846BDE82A
:10CA7000F08110B501220221002000F089FF08B1E9
:10CA8000072810D107220221012000F081FF08B100
:10CA9000072808D100210A22084600F079FF08B1D2
:10CAA000072800D1002010BD022000F085BE000044
:10CAB00070B50024064D06E06868012110F83400C6
:10CAC00003F084FE641C28788442F5D3002070BDF6
:10CAD000002E0020F8B516460C4605460A2A01D25B
:10CAE0000720F8BD03F068FF18B903F02BFF0028FA
:10CAF000F7D1134F202113487D603C70BE60FFF7D3
:10CB0000CEFC0020C7E904000F4E0DE005EBC40089
:10CB10003168009181788DF8011000780B4A6946E0
:10CB200003F0A0FE0028DCD1641EE4B2EED2BDE822
:10CB3000F84005480021064A001D00F087B80000B3
:10CB4000002E00204035002014260200A1E601003E
:10CB50007DDF010072B603F07BF900BF02F0AEFF8B
:10CB60000028FBD111481249401AC408012000EBEB
:10CB7000044010A103F0BEF811480068C00700D0BF
:10CB800000BE022000EB04400EA103F0B3F8BFF397
:10CB90004F8F0B48E43801680E4A01F4E0611143FD
:10CBA0000160BFF34F8F00BFFDE70000F4310200CA
:10CBB0007C310200466174616C206572726F720094
:10CBC000F0ED00E053797374656D207265736574E0
:10CBD000000000000400FA050EB500210091CDE927
:10CBE00001106A4644F20100FFF7B4FF0EBD10B514
:10CBF0008268C368934203D001F082FC002010BD1C
:10CC0000052010BD29B112B1531E134203D00920D3
:10CC100070470E2070470160838000218160C160F1
:10CC20000846704710B58268C3689A1A83889A428A
:10CC300003D801F06FFC002010BD042010BD0000DF
:10CC4000014801F0DABA0000202E00203AB1006855
:10CC50000129426100D000210161002070470720B6
:10CC60007047000038B511480823582241680091E8
:10CC70000F49006801F0A4FF002815D10D4A69464C
:10CC80000D4801F0BFFA04000ED101210A4801F05D
:10CC900034FB0123094A1946074801F086FA064980
:10CCA000012008390870204638BD00001C2602000B
:10CCB0007035002075180200202E0020FFFF7F0035
:10CCC00070B50446007F0D4608B1002070BDA2611A
:10CCD00001F0CCFC401941F10001C4E902012069D6
:10CCE00000B125612146BDE87040002005F004B97F
:10CCF000014600200877012005F0FEB870B50A4E05
:10CD000001460A48B578FFF772FF04464DB100208E
:10CD1000B070711C0122C81D02F096FB08B1FFF72C
:10CD20005BFF204670BD00003C2E0020C83500206F
:10CD3000F0B5244E89B01F460D00044672603FD006
:10CD4000A888296882B22048FFF75CFF002835D107
:10CD5000A889A96882B21C481030FFF753FF002849
:10CD60002CD1202219496846FFF780FB60690690A4
:10CD7000207C00B101208DF814008DF81C70607CBF
:10CD800000B10E208DF81500E0680290A0680390B5
:10CD900020680190606800900A480D4A6946083092
:10CDA00002F01EFB002809D1B0702068401C05D09D
:10CDB00004490122491CC81D02F046FB09B0F0BD20
:10CDC0000720FBE73C2E0020C8350020302602005B
:10CDD0008920020010B501461048FFF723FF040028
:10CDE00019D10F480F4A0178515C19B1001D04F0A8
:10CDF00075F802E00C3003F04BFF60B908490748B2
:10CE00000839FFF7F4FE30B9054901220839044812
:10CE100002F02AFB0446204610BD0000D835002051
:10CE2000442E0020D82D002030B5EFF3108172B6CB
:10CE30000D4A9468012324B10370002900D162B621
:10CE400030BD93604FF0E023D3F88051074C25406C
:10CE50001560C3F88041D3F8844154605A17C3F871
:10CE6000842100220270E8E7E8350020FC06FFBDBF
:10CE70000B498A68002A11D000280FD1EFF31080E7
:10CE800072B60B684FF0E022C2F800314B68C2F86E
:10CE9000043100228A60002800D162B67047000089
:10CEA000E835002070B5054608680C46411C04D0E2
:10CEB00002F003FD206802F063FC6068411C02D0B0
:10CEC000002102F04BFC2968A069C1F82405607DAF
:10CED000227D29681043C1F86C05D4E90012286846
:10CEE000C0F81425C0F80C15207D012814D1A068C5
:10CEF000411C02D0002102F031FCE068411C04D04A
:10CF000002F0DBFCE06802F03BFCD4E90212286886
:10CF1000C0F80825C0F8101570BD70B50546086842
:10CF20000C46411C04D002F0D2FC206802F032FC16
:10CF30006068411C02D0002102F019FC2968A06938
:10CF4000C1F82405607D217D2A680843C2F86C057C
:10CF5000D4E900122868C0F80C15C0F81425207D0B
:10CF6000012814D1A068411C02D0002102F0FFFB6F
:10CF7000E068411C04D002F0AAFCE06802F00AFC60
:10CF8000D4E902122868C0F80825C0F8101570BD51
:10CF900070B5E0B1DAB1002402E0045D2C44A4B223
:10CFA000651C8D4206D21688A642F6D806197678F8
:10CFB0009E42F2D18C420AD2A31C005D9BB200B10A
:10CFC000401E0004000C02D01C188C4201D9002025
:10CFD00070BD138070BD2DE9F0418AB00646002077
:10CFE000ADF814001346102088468DF804000D4655
:10CFF00006AA01A9184665DFA6B398BB9DF80400F0
:10D00000022804D0042807D0102839D10DE00320CD
:10D010008DF81000022003E005208DF81000042098
:10D020008DF81100002404AF0FE007208DF81000E8
:10D030000620F5E73B5D05AA41463046FFF7A8FF0D
:10D04000641CE4B20546022C04D2BDF8140000288A
:10D05000F0D003E0BDF81400002812D080B20644DE
:10D0600000240BE00CE030199DF8042006A9FFF71E
:10D0700028FA48B19DF80400204484B2AC42F2D3AF
:10D0800000200AB0BDE8F0810120FAE770B540B198
:10D090000C4D297839B1044604F052FB28B1002028
:10D0A00070BD0E2070BD082070BDE868062807D24C
:10D0B0000549226801EB8001401C0A60E860EEE748
:10D0C000042070BDC82D00203834002010B558B1A0
:10D0D00003684BB142683AB1044900200124C8609A
:10D0E0000C70C1E9013210BD0E2010BDC82D00200A
:10D0F000002827D0002925D0134A1278002A21D0F1
:10D100000A460188112911D0302907D0322909D0C7
:10D11000332917D1011D104603F0D0BF011D104661
:10D1200004F090B8011D104603F0E8BE8088B2F804
:10D13000CA12884206D1002082F8C8024FF6FF705A
:10D14000A2F8CA0270470000C82D002048B1084A62
:10D15000137843B1D26832B190F8C8222AB11120B5
:10D1600070470E2070470820704700F0C5BF0000D0
:10D17000C82D002038B50288011D04461F2A47D05B
:10D1800016DC102A1ED02B482B4BC01AC0080323D4
:10D1900003EB0040112A2DD0132A33D01B2A44D18F
:10D1A0000979022941D1BDE8384024A102F0A2BD8D
:10D1B000212A31D03B2A39D0562A36D1A0881321D2
:10D1C00077DF11E0A1880022244800F001F908B1BE
:10D1D000FFF702FD072000F0FDFB08B1FFF7FCFCA4
:10D1E000A1881F48FFF7B2FF00281ED0BDE83840D5
:10D1F000FFF7F2BC0B790A8801B01AA1BDE83040F4
:10D2000002F083BD0023A0881A46852180DFEBE76A
:10D2100031F8040B76DFE7E700200090A08869462C
:10D220008DDF002801D0FFF7D7FC38BDA08813217F
:10D2300077DFD9E7F43102007C310200436F6E6E74
:10D24000656374696F6E20526571756573742074BF
:10D25000696D6564206F75742E000000CC3100206C
:10D26000B4270020446973636F6E6E6563746564F0
:10D270002E20636F6E6E5F68616E646C653A20305D
:10D280007825782C20726561736F6E3A203078258E
:10D290007800000010B51A4C0188606810290ED083
:10D2A00011292BD1401E606028D1FFF7E2FB002836
:10D2B00024D02168002921D0BDE810400847D0B90A
:10D2C00000210122084600F063FB08B107280FD1B6
:10D2D00007220221012000F05BFB08B1072807D1DB
:10D2E00004220221002000F053FB20B1072802D0C5
:10D2F000216801B188476068401C606010BD000073
:10D30000C02D002070B506461A481B4A0D46801AEB
:10D31000C0080978032202EB004459B1012922D048
:10D32000022926D1204615A102F0E4FCBDE8704098
:10D3300004F0F6BB204615A102F0DCFC698805F17B
:10D340000E02304600F044F808B1FFF745FC3046C5
:10D3500000F04AF908B1FFF73FFC2046BDE87040F5
:10D360000FA102F0C7BCA989A868BDE8704000F011
:10D3700071B970BDF43102007C31020044697363FD
:10D380006F6E6E65637465642E000000446973639C
:10D390006F7665727920636F6D706C6574652E00B1
:10D3A000436F6E6E656374656420746F2064657688
:10D3B0006963652077697468204E6F7264696320C1
:10D3C0005541525420536572766963652E00000002
:10D3D00050B141802AB15388C380138883809288DA
:10D3E0000281406901F03EBD0E20704730B5144BFC
:10D3F0000D4604000FCB85B08DE80F001ED0EDB1B7
:10D40000A868D8B12146684662DF002814D1207888
:10D410008DF812000120ADF810004FF6FF7060800B
:10D420002868E060686820610020A0802081A868EA
:10D43000606104A8FFF72AFE05B030BD0E20FBE7AF
:10D44000F425020030B5024685B008002DD0002A30
:10D450002BD041884FF6FF74A14226D09388994281
:10D4600023D11588112D14D0392D1ED18188002982
:10D470001BD053898B4218D1C168002915D00121D6
:10D480008DF8001002F110010291D189ADF80C1055
:10D4900008E08B4209D1C168002906D002218DF82D
:10D4A00000104480C2686946904705B030BD30B571
:10D4B00085B00C46054614216846FEF7F0FF20783B
:10D4C00004F10E01002830D1A08801282DD1A079C7
:10D4D0002A78904229D1002217E002EBC20031F8ED
:10D4E0001030022B02D0032B0ED105E001EB4000DF
:10D4F0000089ADF8120007E001EB40000389ADF8A8
:10D500000E304089ADF81000521C207A9042E4D8C9
:10D51000E868002809D06088ADF8020000208DF886
:10D520000000EA6869462846904705B030BD000013
:10D5300070B588B015460E46040012D0202168460A
:10D54000FEF7ADFF19481A49401AC008022101EB45
:10D550000040F42D07D917A102F0CCFB072008B03A
:10D5600070BD0E20FBE76288A2F57F43FF3B18D019
:10D57000154ACDE9022401208DF800002289ADF87A
:10D5800012208DF81010ADF816500022ADF81420BE
:10D5900006968DF8110062886946606901F09AFC70
:10D5A000DDE70AA102F0A6FB0820D8E79C310200C3
:10D5B0007C310200436F6E74656E7420746F6F204F
:10D5C0006C6F6E672E00000035E50100436F6E6ED4
:10D5D000656374696F6E2068616E646C6520696E46
:10D5E00076616C69642E000010B58AB058B341882A
:10D5F000A1F57F42FF3A28D0C18831B304462021EB
:10D600006846FEF74CFF01218DF8201000208DF8B0
:10D6100021000F4ACDE902248DF80010E288ADF810
:10D6200012200222ADF81620ADF814008DF810106B
:10D6300008A88DF81110069062886946606901F0AB
:10D6400049FC0AB010BD0E20FBE70820F9E70000F6
:10D6500035E501002DE9F0410E4605461C481D49FF
:10D660000024401AC008012101EB00480FE0285DAA
:10D67000FFF7B0FB070009D0112FF8D04046224633
:10D6800015A102F03BFB3846FFF7A6FA641CB44232
:10D69000EDD3A81910F8010C0D2804D10A20FFF7CA
:10D6A00099FB1128FAD0324629461548FFF740FF6A
:10D6B00004000BD0112CF6D04046224611A102F0F6
:10D6C0001DFB2046BDE8F041FFF786BABDE8F081BA
:10D6D000F43102007C3102006170705F7561727418
:10D6E0005F707574206661696C656420666F722076
:10D6F000696E646578203078253034782E0000001B
:10D70000CC3100204661696C65642073656E646984
:10D710006E67204E5553206D6573736167652E20CB
:10D720004572726F7220307825782E20000000003C
:10D730000149085C7047000020250200084908B52F
:10D74000085C0090684602F05FF8D0F81005009978
:10D75000C84010F0010000D0012080F0010008BD99
:10D76000202502002DE9FC410646C0074FF00005C8
:10D770000ED0104F00240122385D00950023114681
:10D78000019501F087FF641C042CF4D300F04EF8DF
:10D79000B0070DD5074E0024361D0022305D03234F
:10D7A00000951146019501F075FF641C042CF4D31B
:10D7B000BDE8FC811C250200094908B5085C009001
:10D7C000684602F021F8D0F80425009B0121994019
:10D7D00021EA0203C0F808351140C0F80C1508BD55
:10D7E0001C2502000249085C012102F07AB8000001
:10D7F0001C2502000249085C002102F072B80000FA
:10D800001C250200084908B5085C0090684601F034
:10D81000FBFFD0F804050099C84010F0010000D0CB
:10D82000012080F0010008BD1C25020010B5002475
:10D830002046FFF7D7FF641C042CF9D310BD10B5A8
:10D8400000242046FFF7D6FF641C042CF9D310BD3A
:10D8500010B50246064B4FF0FF3000215C5C94424D
:10D8600001D1084610BD491C0429F7D310BD0000A2
:10D870002025020070B50C4E0C004FF00005306002
:10D880000BD0012000F06AF808B1022004E000206B
:10D8900000F064F800B10B202070706810B9FFF739
:10D8A000E8F80546284670BDC02D002010B50020C0
:10D8B00000F0CAF908B1062806D1012000F0C4F929
:10D8C00008B1062800D1002010BD00002DE9F04766
:10D8D0000D468146FFF7BCFF0446042836D2DFF828
:10D8E00074801B481C4EA8F10C0725B3012D0ED0E7
:10D8F000022D2BD104EB440030444578002D25D077
:10D90000B968002922D02846BDE8F047084704EB53
:10D910004401755C0E44717849B10E4A4FF4804160
:10D92000093A8068FFF7CCF908B987F80390B17815
:10D9300008F80410E2E78068FFF7DAF904EB440125
:10D94000314418F804008D78A842D7D0BDE8F0879C
:10D9500024250200BC2D002008340020042801D218
:10D96000FFF7ECBE00207047042804D00A280CD131
:10D97000002002F081BB05481321408877DF08288A
:10D9800003D0002801D0FFF727B97047CC31002021
:10D9900070B50023042810D20D4D00EB4004012A7D
:10D9A00002D101290CD00022094E00EB4000304486
:10D9B00061B1012906D0022906D00723184670BD9F
:10D9C0000E30C2B22A55F9E74270F7E78270F5E7E8
:10D9D00008340020044A014600201279D20702D000
:10D9E000084600F04DB87047B02D002070B50646CF
:10D9F0001E480024C0E90161B00720D5002501229E
:10DA000011462846FFF7C4FF6D1C0446042D02D2C0
:10DA1000002CF4D013E094B940F2333204211448BE
:10DA2000FFF758F804000AD1FFF742F8040006D1C6
:10DA30000F48104A0021001FFFF708F90446F007BD
:10DA400012D00120FFF78EFE74B909480A4A00215E
:10DA50000C38FFF7FBF8040006D10548074A0121FE
:10DA60000838FFF7F3F80446204670BDB02D0020BB
:10DA70003025020055DD0100D5E80100A9CA0100EA
:10DA80002DE9F05F6E4C054600266078B34618B16C
:10DA900084F801B000F006FF6A4F4FF47A694FF442
:10DAA000C87A4FF00108182D69D2DFE805F00C1391
:10DAB00013384754696E727B727BC5848484848476
:10DAC000B3B6B9BCC5C500F0EDFE3868FFF710F974
:10DAD00006465CE00020FFF795FE00284FF00000AE
:10DAE00008D0FFF77FFE022D02D14FF4E16008E07D
:10DAF000484606E0FFF77EFE022D01D1C82000E077
:10DB00005046410CC0034FF47A72801841F1000175
:10DB1000257052000023FEF765FC01462AE0002034
:10DB2000FFF770FE00284FF0000004D0FFF75AFE08
:10DB30004FF44870E5E7FFF75DFEDFE70020FFF7F1
:10DB400061FE00284FF0000002D0FFF74BFECFE748
:10DB5000FFF750FED4E70020FFF754FE00284FF0F7
:10DB6000000002D0FFF73EFE01E0FFF743FE257004
:10DB700040F6CD4100223868FFF7A2F8064646E09D
:10DB80000020FFF719FE257008E0002051E0257005
:10DB90003DE084F801800120FFF70EFE002240F2F4
:10DBA0006661E8E784F801800120FFF705FE0022A6
:10DBB0004FF40051DFE77868FFF79AF80646D5F191
:10DBC000110000D02EB10220FFF70CFE84F802B045
:10DBD0001DE0012816D980B2C8214843C117C903E6
:10DBE00041EA5041C0034FF47A72801841F10001BC
:10DBF00052000023FEF7F6FB014600227868FFF78B
:10DC00005FF806460220FFF7F5FD84F802803046F3
:10DC1000BDE8F09F00F046FEB9E700F043FEB4E730
:10DC200000F040FE04E000F03DFE0020FFF7E2FDC2
:10DC30000120FFF7DFFDAAE7FFF701FEA7E70000DD
:10DC4000B02D002024250200012104F029BC000091
:10DC50002DE9F84F0546861C00208DF800009146FE
:10DC60000F464FF0010A6846FFF7DEF81B4C04F23E
:10DC70001C4860683860D4E90101194F401A3968BE
:10DC8000081A0EE00121404600F0DFFF00F034FEEC
:10DC90000146404600F0D9FFD4E90101401A396835
:10DCA000081A401C8642EDD8B9F1000F03D00520B8
:10DCB00065F3891002E0062065F39F5061683A68B9
:10DCC000114004EB8101C8606068304460609DF8D9
:10DCD0000000FFF7CDF85046BDE8F88F98370020D8
:10DCE0007C2E002070B50D4604460A2902D10D2174
:10DCF000FFF7F8FFA0682268411CA1601554D4E921
:10DD00000101814204D32046BDE8704001F0C9BB47
:10DD100070BD0000044881684068814201D1012043
:10DD2000704700207047000098370020034630B548
:10DD3000074800210478426806E000BF02EBC100FA
:10DD400005789D4203D0491CA142F7DB002030BD7D
:10DD5000002E002000780221FFF7B8BD05494FF0E2
:10DD6000FF32082841F8202002D3084480F85220CE
:10DD70007047000064340020F0B54FF0FF3512B159
:10DD80000023082601E008230C260C4C05E000BF08
:10DD900054F823707F1C04D05B1CB342F8D3284690
:10DDA000F0BD26185DB286F8305044F82310002AE2
:10DDB000F5D1E11881F85200F1E700006434002049
:10DDC0000249084490F93000704700006434002094
:10DDD00030B589B00D46044620216846FEF75FFB4A
:10DDE00094F8C602002300EB8001C1EB801094F888
:10DDF000C51204EB400041B1491EC9B201EBC1019B
:10DE000000EB4101498A491C00E0C188008961F3A7
:10DE10000F0360F31F4303208DF800000548CDE990
:10DE20000204054804932A466946806801F052F8C6
:10DE300009B030BDA9E00100C82D002070B5084C24
:10DE4000050009D010342168002907D00868206037
:10DE5000496828468847F6E70834F4E770BD0000B3
:10DE600050340020054A012120B1012805D19170CC
:10DE7000FFF7E4BF51700020FAE7704750340020EC
:10DE800010B5D0E90234D1E90220D11AA04101D362
:10DE9000012010BD002010BD10B5024600201388DF
:10DEA00006E0546834F810408C4203D0401C80B225
:10DEB0008342F6D810BD000001460148FFF7F7BACB
:10DEC000CC3100202DE9F04389B00F46054691463C
:10DED00020216846FEF7E3FA95F8C60295F8C54298
:10DEE00000EB8001C1EB801005EB400604EBC400A1
:10DEF00006EB40013279601C0A31904232D108AB06
:10DF00000022284600F09CFC78B310E0401EA0429E
:10DF100001D1002004E004EBC40006EB40001C30FB
:10DF20008046024608AB284600F08AFC90B10020EB
:10DF3000387004208DF8000008984A46CDE9035057
:10DF40000C4802900C486946806800F0C3FF09B095
:10DF5000BDE8F08395F8C5024146401C641C85F875
:10DF6000C502E4B23079A042D0D801203870002038
:10DF7000EDE70000A9E00100C82D002070B50024E5
:10DF80000F4D10E0686800EBC406307802F0D2FC58
:10DF90007178012901D0012100E000214140307851
:10DFA00000F034FA641C28788442EBDBD5E90401E4
:10DFB000084303D0BDE8704003F0BABF70BD000055
:10DFC000002E002030B59FB00C4605467C216846E7
:10DFD000FEF765FAADF8024003208DF80000044812
:10DFE00001954168002901D0684688471FB030BDBF
:10DFF000C82D00202DE9F041044690F8C60288465D
:10E0000000EB8001C1EB801004EB40061746304660
:10E0100003F096FB050042D0D4F8CC0206283ED28D
:10E0200004EBC0107622A0F8D272D4F8CC023146AC
:10E0300004EBC01000F53570FEF718FA0026B8F1B1
:10E04000000F06D0D4F8CC0204EBC01080F8D062E8
:10E0500006E0D4F8CC12022004EBC11181F8D00202
:10E06000D4F8CC0204EBC010C0F84C53D4F8CC0266
:10E070000C4D401CC4F8CC02E96888420FD12746F9
:10E08000002407E007EBC41101F53470D1F84C13FC
:10E090008847641CE8688442F4D3C7F8CC62BDE8C2
:10E0A000F0810000C82D0020F0B515469FB0002279
:10E0B00081F8C822074691F8C6020C4600EB8002A0
:10E0C000C2EB801001EB400003F03AFB060009D0E0
:10E0D0007C2208496846FEF7C9F9ADF80250684647
:10E0E0000197B0471FB029462046BDE8F040FFF732
:10E0F00069BF000050250200F0B50D4689B0044606
:10E100004FF4BA61FEF7CBF920216846FEF7C7F954
:10E11000154E2946B06800F0A5FE002821D1A4F8CC
:10E12000CA52C4F8CC0284F8C70284F8C60284F844
:10E13000C5020E4801272A460068206002208DF89B
:10E140000000ADF810702068CDF812000848CDE945
:10E1500002046946B06800F0BDFE002801D184F8D1
:10E16000C87209B0F0BD0000C82D0020383400206E
:10E17000A9E0010010B50021024800F071FD80F314
:10E18000100010BDB43B00204FF480328A4001687B
:10E19000C1F848230068C0F8082370474FF4A07204
:10E1A00002EB810189B200F0A1B92DE9F0410546E9
:10E1B0000E464FF4A07000EB860081B228684FF441
:10E1C0008034B440984622F07F47C0F8084328685E
:10E1D000C0F84843286802F03AF8286800EB860047
:10E1E000C0F840752868C0F84443B8F1000F02D069
:10E1F0002868C0F80443BDE8F0810068D0F8040541
:10E200007047000070B54379234C44F823204279CD
:10E21000231D03EBC202224C1579204A121BD4089D
:10E220002DB10825022000EB04401EA130E0056856
:10E230000A88C5F8082590F904208978002A4FEA51
:10E24000411104DB02F1E02282F8001405E002F043
:10E250000F0202F1E02282F8141D90F9041001224D
:10E26000002909DB01F01F0502FA05F549098900BB
:10E2700001F1E021C1F800514179002503EBC10112
:10E280000A71417943F83100032000EB04400EA1EC
:10E2900001F030FD284670BD582E0020DC31020010
:10E2A0007C31020052544320696E7374616E636561
:10E2B00020616C726561647920696E697469616C52
:10E2C000697A65642E0000005254433A20696E69F1
:10E2D0007469616C697A65642E00000090F904002D
:10E2E000002809DB00F01F02012191404009800055
:10E2F00000F1E020C0F8001270470A46022100F049
:10E300007BB84FF4827100F0F1B800680121016020
:10E31000704700680121416070472DE9F05F0746B2
:10E320000C464FF4A07000EB84001FFA80FA3868A6
:10E330004FF48036A6409B4622F07F45C0F84863E4
:10E340003868C0F808633868D0F8048500EB8402A8
:10E35000D2F84095C2F840855146386801F077FF01
:10E36000A9EB080020F07F40012806D1102002F020
:10E3700025FA5146386801F06AFF3868D0F80485FC
:10E38000C0F84463A5EB080121F07F4138680129FA
:10E3900000EB840010D0C0F840553868D0F8041560
:10E3A0006FF07F4C6A1A521E22F07F42ACEB0B03D7
:10E3B000934217D362B118E06D1CC0F8405510208D
:10E3C00002F0FCF93868D0F8040540450AD10CE0A9
:10E3D00000EB84006D1CC0F840553868D0F8040587
:10E3E000884202D00D20BDE8F09F01223146384618
:10E3F00000F002F80020F6E70368C3F84413002A8F
:10E4000002D00068C0F80413704700002DE9F84FEF
:10E410000E463449804601EB5001C007097801D00F
:10E420000F0901E001F00F074FF0000942460120FB
:10E430004946FEF708F8DFF8B0A004460D46052F60
:10E440004ED2DFE807F003161B282C00002E47D021
:10E450000121404603F086FC8DF800906846FEF7E7
:10E46000E3FC5046D0E904120C431543CAE90445C5
:10E4700032E00EB1022114E0002112E04EB103217E
:10E48000404603F06FFC4046BDE8F84F012103F021
:10E49000F7BF012105E0002E22D1042101E02EB1B9
:10E4A00003214046BDE8F84F03F05CBC0021404624
:10E4B00003F058FC0021404603F0E2FF8DF8009085
:10E4C0006846FEF7B1FC5046E243D0E904341A40F6
:10E4D00024EA0501CAE904219DF80000FEF7C8FC02
:10E4E000BDE8F88F40350020002E002010B50068F0
:10E4F00042581AB101F0ABFE012010BD002010BD42
:10E50000826883881A4003689A5C0A708168491C93
:10E5100081607047C26883881A4003689954C16853
:10E52000491CC160704710B50446C0B2FEF752FCEA
:10E53000204610BD0969002900D008477047000037
:10E5400070B508880D46A0F52061773916D10C48C2
:10E550000C49401AC108032000EB01440AA12046DF
:10E5600001F0C8FBA88810A1C01E82B20D48134656
:10E5700002802046BDE8704001F0C7BB70BD0000BE
:10E58000F43102007C310200415454204D54552096
:10E5900065786368616E676520636F6D706C657424
:10E5A00065642E00B0270020426C65204E55532034
:10E5B0006D61782064617461206C656E6774682099
:10E5C00073657420746F20307825582825642900DD
:10E5D00010B50949094800F0BAFB08B1FEF7FCFA8A
:10E5E000F721064800F0A7FB002803D0BDE8104043
:10E5F000FEF7F2BA10BD000041E50100E431002051
:10E6000070B50D4601F11004C98A102901D90920FD
:10E6100070BD01F08CFC686030B1E2880023A16815
:10E6200001F0EBFC002070BD042070BD70B50D46FC
:10E6300001F1100489690988102901D9092070BDE8
:10E64000891C01F074FC686068B100230222A16893
:10E6500001F0D3FCA068E16802230288686801F039
:10E66000CCFC002070BD042070BD000010B50B482C
:10E67000FFF7C3FD094A083AD2E90434C018D2E9C9
:10E68000063244F10001C31A71EB020204D24FF0CA
:10E690008072801841F1000110BD0000202E002082
:10E6A00010B5C0B2FFF742FB0446007802F042F911
:10E6B00001466078012801D0012000E0002090EAA6
:10E6C000010F08D00449D1E90401084303D1BDE892
:10E6D000104003F02DBC10BD002E00202DE9FC5F82
:10E6E0000E008346DDE90C47C6F1000098469246CD
:10E6F000814600D40846012503E000BF90FBFAF0F4
:10E700006D1C5045FADAA84500D9454624B1002EC3
:10E7100001DB780700D5641EB80702D5B8F1000FF9
:10E720000AD0F80708D13CB1A54205D220215846AD
:10E73000641EFFF7D7FAF6E7002E02DA4E462D21C7
:10E7400002E0780703D52B215846FFF7CBFA07F0F4
:10E75000030002280BD1B8F1000F08D13CB1A5424B
:10E7600005D230215846641EFFF7BCFAF6E7CDE922
:10E770000047434652463146584603F027FEBDE85F
:10E78000FC9F000070B50D46044600684FF4887188
:10E7900001F0CAFF4FF49071206801F0C5FF4FF4FB
:10E7A0009271206801F0C0FF4FF4A271206801F05F
:10E7B000BBFF4FF4AC71206801F0B6FF206812492E
:10E7C000C0F804132068690740F30730090E0028D9
:10E7D00004DB00F1E02080F8001405E000F00F00F9
:10E7E00000F1E02080F8141D206840F30730002875
:10E7F00009DB00F01F02012191404009800000F177
:10E80000E020C0F8001170BD100342000246002055
:10E810001268530713D502F00300012802D0022822
:10E820000CD105E0C2F383100B68801C184404E08F
:10E830000223086803EB92521044086001207047DD
:10E8400010B509892AB1D088491C814218D100200D
:10E8500010BD90F8C62202EB8204C4EB821200EBDA
:10E86000420212899142F2D0491C198090F8C612D6
:10E8700001EB8102C2EB811100EB4100008902E053
:10E880001980D088401E5880012010BD007DC0F343
:10E89000C100012803D0032801D0002070470120C7
:10E8A000704700000A4810B5807860B1002401E08C
:10E8B000022C06D02046FEF795FF641C042CF7D3EB
:10E8C00010BD0324F6E7BDE81040FEF7AFBF00001F
:10E8D000B02D002003480179C90702D00078FFF766
:10E8E000CFB87047B02D0020F7210180172141805B
:10E8F00000210171417170472DE9FF410026244834
:10E9000000F0A0F92248001F074600F09BF9214CB7
:10E910002149A06800900D6800E0009869462840F1
:10E9200004EB80000C30FFF771FF0028F5D101AA3D
:10E93000009901EA050304EB8303491CDB6842F8F4
:10E940002030401C00910228F2D3019800F003000F
:10E9500001280BD0022810D10198032101EB90501F
:10E960000099BDF80A6001EB900005E00198BDF840
:10E970000A60C0F3831008440090384600F05FF945
:10E9800008B10098A06004B03046BDE8F0810000F6
:10E99000B03B0020983700207C2E00208AB04FF436
:10E9A0008041002001F028FA08B1FEF715F901F0C6
:10E9B00077F8FEF757F908B1FEF70EF91822364935
:10E9C0006846FDF753FD3548069035494FF4807091
:10E9D000CDE9070109900723324A06A96846FEF7E8
:10E9E000A7F908B1FEF7F8F82F490120FEF7FEFF5E
:10E9F00008B1FEF7F1F869460020FEF73BFF08B1C9
:10EA0000FEF7EAF82A4C2948CDE9000400256846BB
:10EA1000FEF75CFB08B1FEF7DFF801F0F7FA08B18A
:10EA2000FEF7DAF801F082FD08B1FEF7D5F8694685
:10EA30000120009501F01CFC08B1FEF7CDF86846F6
:10EA400001F0ACFC08B1FEF7C7F8FFF7C1FD1948AB
:10EA500000901948CDE9010469461848FEF7C6FC44
:10EA600008B1FEF7B9F803F02FF815A0FDF7C6FFBF
:10EA70001C481D49401AC008032101EB00401BA19E
:10EA800001F038F903F04CF801F018F80028FBD138
:10EA900001F0D0FAF8E7000004250200CC2F002096
:10EAA000CC3000209D1F020069D90100B9DE0100B1
:10EAB000842D002005D30100F90E0200CC31002086
:10EAC000424C4520554152542063656E7472616C0E
:10EAD000206578616D706C65207374617274656413
:10EAE0002E0D0A00F43102007C310200424C452018
:10EAF000554152542063656E7472616C2065786173
:10EB00006D706C6520737461727465642E00000012
:10EB10002DE9F047C5881E1DB6FBF5F78946B6FB03
:10EB2000F5F1044605FB176C407916686843DDF87B
:10EB300020A0F718001F874200D9C61A166001E00E
:10EB40002468491E0029FBD1A5EB0C078846B74273
:10EB500016D818E004EB0C00001D09EB0803BAF10D
:10EB6000000F3A4602D00146184600E01946FDF76C
:10EB70007DFC2468F61B4FF0000CB844B54201D967
:10EB8000374600E02F46002EE4D1BDE8F0870000B4
:10EB900030B5024651B101F043F90021074C08E0BD
:10EBA00034F821301568AB4202D11160002030BD2D
:10EBB000491C8142F4D3052030BD00000000000054
:10EBC00010B531B1B2FBF3F403FB14241CB10920DE
:10EBD00010BD0E2010BD0160002141608160828166
:10EBE000C381084610BD70B50C460546FDF712FB03
:10EBF000002802D021882868084470BD10B50A8812
:10EC000049888A4203D1FDF747FB012010BD00204F
:10EC100010BD70B50C460546FDF721FB002802D05B
:10EC200061882868084470BD10B50A8849888A42FE
:10EC300003D1FDF70BFB012010BD002010BD00210A
:10EC400000F009B8012100F010B808B56A46FDF7D8
:10EC500078FB009808BD08B56A46FDF758FB08BD6B
:10EC600008B56A46FDF73AFB08BD08B56A46FDF7E8
:10EC700041FB009808BD08B56A46FDF76FFB009898
:10EC800008BD38B5044600258DF800506846FEF7EB
:10EC9000CBF821686268086890420ED9401E08606F
:10ECA0000178238AE26801FB0325227A2168101A81
:10ECB000C0B20A79824200D208719DF80000FEF7C6
:10ECC000D7F8284638BD38B5054600208DF8000035
:10ECD0000C466846FEF7A8F8E868298A201AB0FBB7
:10ECE000F1F12A681068431C136001709DF8000060
:10ECF000FEF7BEF838BD10B530B1017A426803683E
:10ED0000891AC9B21A6006E00E2010BD03681A689D
:10ED1000541C1C601170491EC9B2F7D20068002152
:10ED20000171084610BDC20800F007030120895C8C
:10ED300098400840704728B1A1F11702E12A03D397
:10ED4000072070470E20704741800020704710B5A3
:10ED500060B10161F72120F8021B20F8021BFB21A2
:10ED600000F8021BFFF7C0FD002010BD0E2010BDF3
:10ED70007CB585880C46002D33D1018800261029EA
:10ED800006D0112909D03A290BD055292ED129E0D6
:10ED90000146204602F04EF928E0A01DFFF7A4FD31
:10EDA00024E02246408934F8061F814200D80846F4
:10EDB0006080172800D217206080106978B16079D0
:10EDC00068B11849D1E90001CDE90001ADF8025060
:10EDD0006088ADF80400136969461046984766716B
:10EDE00026717CBD0146204602F0D6F9A07A0028A3
:10EDF000F7D0E1882846A5DF012580B11128F0D0A1
:10EE000001F072FC02460848084902B0401AC008E6
:10EE100005EB0040BDE8704005A100F06FBFA67291
:10EE2000E5727CBDCC250200843102007C310200F9
:10EE300073645F626C655F67617474635F65786358
:10EE400068616E67655F6D74755F72657175657316
:10EE50007428292072657475726E65642025732E7E
:10EE6000000000002DE9F0410F4604004FF00005BE
:10EE70000DD002F039FC39462046FFF70DF8218805
:10EE800081421ED1002005464FF6FF7609E00E2094
:10EE9000BDE8F081626832F81020B24206D1401C11
:10EEA00080B28142F6D8206901F08EF800202188D6
:10EEB0000BE0626832F81020B24204D1616821F898
:10EEC00010702846E4E7401C80B28142F1D804204B
:10EED000DEE700002DE9F04791460D4604004FF0B3
:10EEE000000742D0EDB302F0FFFB49462046FEF793
:10EEF000D3FF2978062902D22188814202D1072036
:10EF0000BDE8F087A16800EB800601EB860001F008
:10EF100018F930B14946284602F052FC08B138468B
:10EF2000EEE72978DFF8488058F821202AB12069D7
:10EF3000B8B1294690470028E2D1A068294600EBE5
:10EF4000860001F01DF9070006D0297858F8210045
:10EF500010B1686801F01BF8A068494600EB860014
:10EF600000E002E002F028FBD9E70E20C8E700002D
:10EF7000DC250200F8B505000C4620D0002C1ED080
:10EF80002888112806D0A0F130011F2902D9503855
:10EF90001F2814D8AE8820463146FEF77DFFADF815
:10EFA0000000218881420AD02988112908D0A1684F
:10EFB00000EB800001EB8000314602F0FDFAF8BD65
:10EFC00062684FF6FF7122F810106946E06801F0A0
:10EFD000D7F8F8BD2DE9F041044600F1140700F11F
:10EFE0000A05867C007A86B001F10208002814D058
:10EFF0008ADF14216846FDF752FA33462A4639461D
:10F0000040468BDF05218DF800100190002804D0C8
:10F01000A16A002901D06846884706B0BDE8F081A2
:10F020004FF4C8710182062141811821818100219C
:10F03000C1817047017D074A82615210C26121F08F
:10F0400018010022028441F004010175012141757B
:10F0500070470000A0860100F0B520B11AB1032965
:10F0600003D00720F0BD0E20F0BD04790346051D36
:10F070000CB10420F0BD00211688084633F8217039
:10F08000B742F7D0491C11F0FF01F7D003EB840120
:10F09000641C2C7012680A60F0BD18B10021417127
:10F0A000084670470E20704710B50B46040002D08A
:10F0B000980702D009E00E2010BD580705D4D806E5
:10F0C00003D4180701D4072010BD2046FFF7E5FF41
:10F0D000580701D501206071A271002010BD70B5E4
:10F0E0000D46040010D0002626606660A262EDB1D5
:10F0F00028792072287BA074296839B1142204F180
:10F100001400FDF7B3F904E00E2070BD2046FFF7B0
:10F1100091FFA86830B10168C4F80A104068C4F8CB
:10F120000E0009E02046FFF77BFF05E0FFF782FFB6
:10F130002046FFF775FF267204F12C00E0641F20C3
:10F14000A4F85000002070BD2DE9F04F044689B0AE
:10F15000002088460746069014216846FDF79FF96F
:10F1600004F1140004902046FFF790FB010004F125
:10F170004C00059011D002208DF80000CDF80480DD
:10F18000A16A684688470020059989DF41462046E4
:10F19000FFF720FF09B0BDE8F08FA07900210791AB
:10F1A0006179834621B301210691824694F8049047
:10F1B0000026B8F81C003546089012E004EB8502E2
:10F1C000D8F818000899FDF706FF28B1761CF6B2AA
:10F1D000BAF1000F0DD002E0BAF1000F06D16D1C9C
:10F1E000EDB24D45EAD3BAF1000F02D04E4501D041
:10F1F00009E046B19DF8080040F004008DF80800D1
:10F2000001207F1C0790CDF80480BBF1000F02D0D5
:10F210000698874203D0079830EA0B0007D00020F9
:10F220008DF8000041462046FFF7D4FE02E003209F
:10F230008DF80000A16A09B1684688470020059949
:10F2400089DFA7E770B50D46014601F108020C1DE4
:10F2500028460988143586B010291ED01B2907D0EE
:10F260001D292DD106B01146BDE87040FFF76CBFD7
:10F27000064614216846241DFDF711F9207801285F
:10F280001ED1B06A00281BD004208DF80000049520
:10F2900020788DF80400B16A10E006461421684613
:10F2A000FDF7FDF806208DF80000201D0190208854
:10F2B000ADF808000495B16A002901D06846884776
:10F2C00006B070BD30B585B0040025D01421684665
:10F2D000FDF7E5F88ADF2046FFF7D8FA012528B1C7
:10F2E000A16A19B18DF800506846884704F14C01B5
:10F2F00004F1140089DF044608280FD074B10848CF
:10F3000008492246401AC00805EB004006A100F05B
:10F31000F5FC204605B030BD0E20FBE70020F9E7E4
:10F32000943102007C31020073645F626C655F6738
:10F3300061705F7363616E5F737461727420726574
:10F340007475726E656420307825780000F1804015
:10F350000068002800D00120704708B500F1804007
:10F36000002101600068009008BD000070B50D4CE0
:10F370000125207808B185260EE00020A06060609D
:10F380002061E060084801F0F3F9064601F01AF93F
:10F3900008B901F0D7F9257001F0CCF900B1A570DA
:10F3A000304670BD5034002065DE010038B50025C0
:10F3B0008DF800506846FDF737FD084CE068401EA8
:10F3C000E060E06828B901F0B5F910B901F0DEF9A4
:10F3D000A5709DF80000FDF74BFD38BD50340020AE
:10F3E000F0B505460478154889B0164640F8242043
:10F3F000124A08690832A2F10C0742F82400487F3B
:10F40000385520226846FDF731F804942878385C96
:10F4100048B10EB10A4A00E000226946281D01F0F9
:10F420004FFC09B0F0BD0EB1064A00E0002269466B
:10F4300005F10C0001F0F8FAF3E70000DC2D0020E4
:10F44000892202002D21020030B40378054CE35CD0
:10F450001BB130BC001D01F069BC30BC0C3001F0A8
:10F460004DBB0000D82D002030B40378054CE35C80
:10F470001BB130BC001D01F0DBBC30BC0C3001F016
:10F48000B3BB0000D82D00200FB408B503990029A4
:10F4900004D004AA00926A4600F00FF801B05DF8AB
:10F4A00014FB10B582680446002A05D0D4E9040391
:10F4B000216898470020A06010BD2DE9FC479146C7
:10F4C0000C00804676D014F8011B39B125290ED0E6
:10F4D0004046FEF707FC20780028F4D198F80C008D
:10F4E000002867D04046BDE8FC47FFF7DABF0020A0
:10F4F000012221782B291BD02D2902D0302908D1B7
:10F5000002E040F0010001E040F00200641C002A2B
:10F51000EFD100252A290ED02178A1F130020A2A44
:10F5200011D205EB850201EB4205641C303DF1E789
:10F5300040F00400EAE7D9F800100B1DC9F80030CC
:10F540000968641C0D44217800232E290BD114F87E
:10F55000011FA1F130020A2A05D203EB830201EB5D
:10F560004203303BF3E76C290DD068290BD06929A1
:10F5700021D00BDC252918D0582931D063290ED091
:10F58000642915D117E014F8011FECE7702969D040
:10F59000732932D075291BD0782909D120E0D9F8F8
:10F5A0000000011DC9F8001001784046FEF79AFBE3
:10F5B000641C90E76CE0D9F800100A1DC9F800201F
:10F5C0000968CDE900500A224046FFF787F8EFE7C7
:10F5D000D9F800100A1DC9F8002009680A2206E0BF
:10F5E000D9F800100A1DC9F8002009681022CDE9D9
:10F5F0000050404602F0EAFEDAE7D9F80010002792
:10F600000A1DC9F800200E68C00705D112E0404667
:10F61000761C7F1CFEF766FB31780029F7D104E0E9
:10F62000202140466D1EFEF75DFBBD42C0D9002D76
:10F63000F6D1BDE74EB13046FCF73CFF074604E08B
:10F64000202140466D1EFEF74DFBBD4206D9002D20
:10F65000F6D103E04046761CFEF744FB31780029E2
:10F66000F8D1A5E7D9F80000011DC9F80010056818
:10F6700030214046FEF736FB78214046FEF732FB4C
:10F6800008200021CDE90001034610222946B0E7F9
:10F69000BDE8FC872DE9FF411C46DDE90A781546E7
:10F6A0000E46684600F0B0F846EA450141EA84019A
:10F6B00041EA072242EA0841009A00EB8200C0F8C2
:10F6C0000017BDE8FF812DE9FF411C46DDE90A78FE
:10F6D00015460E46684600F0A5F846EA450141EA9F
:10F6E000840141EA072242EA0841009A00EB8200C5
:10F6F000C0F80017BDE8FF812DE9FF411C46DDE998
:10F700000A7815460E46684600F09AF846EA450122
:10F7100041EA840141EA072242EA0841009A00EBEB
:10F720008200C0F80017BDE8FF812DE9FF411C46AB
:10F73000DDE90A7815460E46684600F08FF846EA7D
:10F74000450141EA840141EA072242EA0841009A60
:10F7500000EB8200C0F80017BDE8FF811CB5002255
:10F760000B46009211460192FFF7C6FF1CBD1CB567
:10F7700000220B46009211460192FFF7D6FF1CBDF6
:10F780001CB5002100910B46012201911146FFF7A3
:10F79000B3FF1CBD1CB5002100910B460122019155
:10F7A0001146FFF7C2FF1CBD13B50C46684600F0BA
:10F7B00039F8009900EB8101D1F8002722F440329A
:10F7C000C1F80027009900EB8100D0F8001741EA4A
:10F7D0000441C0F800171CBD3CB50A4CD4E9003404
:10F7E000CDE900346B46441808E000BF53F8201000
:10F7F000D1F8205520C2C1F82055401C8442F5D8CC
:10F800003CBD0000042602000168202902D24FF00E
:10F81000A040704701F01F010160014870470000DF
:10F82000000300500168202902D24FF0A040704729
:10F8300001F01F0101600148704700000003005003
:10F840000168202902D24FF0A040704701F01F014B
:10F850000160014870470000000300500168202942
:10F8600002D24FF0A040704701F01F010160014833
:10F87000704700000003005042094FF0000102D021
:10F88000012A05D102E04FF0FF3101E040F2FF31E3
:10F8900000F01F00012282400A4201D0012070477F
:10F8A0000020704701B56846FFF7BCFFD0F810058F
:10F8B0000099C84000F0010008BD01B56846FFF797
:10F8C000BFFF009A01219140C0F8081508BD01B59D
:10F8D0006846FFF7C3FF009A01219140C0F8081560
:10F8E00008BD38B501240090684631B1FFF78CFFA0
:10F8F00000998C40C0F8084538BDFFF785FF009996
:10F900008C40C0F80C4538BD034908B508440021B7
:10F9100001600068009008BD006000400249405846
:10F92000012800D0002070470060004030B5154A23
:10F9300001460020D2F8104423460AE0DB681D7916
:10F94000854205D1401C0A28F6DB4FF0FF3030BD60
:10F950001B68002BF2D1431CF9D0CB681871D2F888
:10F96000103443B1DB68CC681B682360D2F81024E4
:10F97000D268116030BDC2F81014C96800220A6054
:10F9800030BD0000983700207047FCF781BE7047FB
:10F9900008B5034A00924023024A00F005F808BD6A
:10F9A000FD1B020000360020F0B595B01C46154640
:10F9B0000F4608461A9E00F003FB182109A8FCF721
:10F9C0006EFD0E96CDE909540023082203A938469E
:10F9D00000F00BFB05980690BDF81000ADF81C0078
:10F9E000BDF81200ADF81E0000208DF8210003982C
:10F9F000082600F00300012802D0022818D032E0C7
:10FA000003983346850AC0F3C2008DF8200003989E
:10FA10000FA9C0F38314A200384600F0E6FA09A843
:10FA2000009006AB22460FA9284600F025FA1AE0FE
:10FA30000398840DC0F3C2008DF82000082C01D279
:10FA4000254600E0082533462A460FA9384600F02F
:10FA5000CCFA2E44641B09AB06AA29460FA800F075
:10FA600073F9002CEAD1384600F0B0FA15B0F0BDB9
:10FA70000A4A012902EBC00007D0022907D0032956
:10FA800007D0042907D000207047022070470420C7
:10FA90007047007970474079704700007C31020060
:10FAA00010B5FFF772FF04210348FFF73FFF02493B
:10FAB0000120C968487110BD6C3102002DE9F04F7A
:10FAC0008DB0FEF727F918B100200DB0BDE8F08F1A
:10FAD0007E4C4FF0000BC4F818B4BFF34F8F7C4935
:10FAE000A06802900D68D846284004EB80000BE027
:10FAF000D4F8180470B961680298814201D8A160F5
:10FB0000E2E7284004EB80000C3002A9FEF77EFEFD
:10FB10000028EDD1002005AA029901EA050304EBB3
:10FB20008303491CDB6842F82030401C0291022804
:10FB3000F2D3059800F00300022802D001284DD02E
:10FB4000AAE005985022810D8946B2EB905F00D85B
:10FB500050210E4666F39F50059008315D4800F035
:10FB6000E6F9070078D000F02BFA4346082205A9F1
:10FB7000384600F042FA029908F1080A2940681A4A
:10FB80008000001D864222D9504D0C3530B1C2B2E2
:10FB900004EB8101301A90460C3104E02946F2B2A0
:10FBA000002590462846C6B25346384600F025FA4E
:10FBB0000AEB080325B132462946384600F01DFA03
:10FBC000029909F1030001EB900002903BE004EB85
:10FBD00081015346324638460C31EFE70598C0F3B1
:10FBE0008310062800D30620059960F38911C1F31C
:10FBF0008310801C05918100364800F098F90700B9
:10FC00004AD000F0DDF94346082205A9384600F045
:10FC1000F4F908F1080800260FE00298434600EACC
:10FC20000501401C04EB81010290042238460C318E
:10FC300000F0E3F908F10408761C0598C0F383107E
:10FC4000B042EAD847B1D4F81054D4F8180478B1C7
:10FC5000384600F0BBF934E01EE0E868407901283E
:10FC600004D12A682846394612689047E868056832
:10FC7000002DF2D1384600F0A9F98DF800B06846A1
:10FC8000FDF7D2F8D4F8180408B90298A0609DF8DE
:10FC90000000FDF7EDF814E0D4F8104405E0216809
:10FCA000204689688847E0680468002CF7D10A4834
:10FCB0000A49401AC008022101EB004008A100F0E7
:10FCC00019F8FEF727F880F00100FEE698370020CB
:10FCD0007C2E002028320200F43102007C31020028
:10FCE0004261636B656E647320666C7573686564EE
:10FCF0000000000000231A4602F04CB808B50123AA
:10FD000000926A4602F046F808BD1CB5CDE9002312
:10FD100002236A4602F03EF81CBD3EB5069C8DE803
:10FD20001C0003236A4602F035F83EBDF0B587B0EB
:10FD30000DF1300C9CE8F0008DE8FC0006236A46CB
:10FD400002F028F807B0F0BD2DE9F0470E468046D6
:10FD50001C469246082940D894F80C900020207345
:10FD60001946104601F0D0FB0025B54206D218F81E
:10FD700005201BA12046FFF787FB03E01AA12046C0
:10FD8000FFF782FB6D1C082DEFD318A12046FFF76B
:10FD90007BFB0025B54212D218F805707E2F08D8DB
:10FDA000FCF760FB0068C05D10F03E0F01D03A46E2
:10FDB00000E02E220EA12046FFF766FB03E00DA116
:10FDC0002046FFF761FB6D1C082DE3D3012221467D
:10FDD000504601F07BFB84F80C90BDE8F0870000F2
:10FDE0002025303278000000202020007C00000018
:10FDF0002563000020000000064910B500200870AF
:10FE0000054800F0E1F8002803D1044800F011FA99
:10FE1000002010BD9837002028320200E827020099
:10FE200002480349401AC00870470000143202001B
:10FE30007C31020013B56846FEF7AAFE08B1002027
:10FE40001CBD0248009950F831001CBD7C310200F5
:10FE500070B508480125D0F81044057007E0E06847
:10FE600045712168204649688847E0680468002C8D
:10FE7000F5D170BD983700202DE9FF4781460C9DD4
:10FE800000200C462F7B28739846164629461846B4
:10FE900001F03AFB072E42D2DFE806F004090F1604
:10FEA0001F2A360049462846FFF7EEFA37E0494652
:10FEB00028462268FFF7E8FA31E0D4E900234946F2
:10FEC0002846FFF7E1FA2AE0A0680090D4E9002371
:10FED00049462846FFF7D8FA21E0D4E90201CDE9E6
:10FEE0000001D4E9002349462846FFF7CDFA16E081
:10FEF00004F1080007C88DE80700D4E9002349464B
:10FF00002846FFF7C1FA0AE004F108000FC88DE89F
:10FF10000F00D4E9002349462846FFF7B5FA00222E
:10FF20002946404601F0D2FA2F73BDE8FF872DE93C
:10FF3000F041058A80462D1F4819C01CB0FBF5F022
:10FF4000C6B24046FEF79DFE041E19D00020207167
:10FF500001206071E58000272546761EC4F80080E8
:10FF60000BE04046FEF78DFE60B16179491C61717E
:10FF7000286005467F1CC0F80080B742F1D32046B8
:10FF8000BDE8F081204600F002F80020F8E72DE9F6
:10FF9000F041457901466B1E002201E00968521CC0
:10FFA0009A42FBD30F680146002605E038460C68EC
:10FFB000FEF789FE2146761CAE42F7D3BDE8F081FC
:10FFC0000121001DFEF741BEFEF795BE10B50446A7
:10FFD0000121001DFEF74FFE10F0FF0F04D1204657
:10FFE000BDE81040FFF7D3BF10BD1CB50192012240
:10FFF000009201AAFEF78CFD1CBD1CB501920022E7
:020000040002F8
:10000000009201AAFEF784FD1CBD0000064910B550
:1000100000204870091D0860BFF35F8F0349044842
:1000200000F0F4FA002010BD642E002080260200AB
:10003000F435002008B500208DF800006846FCF774
:10004000F3FEF1EE100A20F09F00E1EE100ABFF37C
:100050005F8F08494020C1F880029DF80000FCF73E
:1000600007FF00F0AFFA08B141DF08BD20BF40BF75
:1000700020BF08BD04E000E070B504460C48012133
:10008000FEF7EEFDBFF35F8F0025002809D10120A8
:10009000074E042C08D0311F4A781AB1BFF35F8F86
:1000A000356070BD0C70487001F0E0FDF6E70000AF
:1000B000682E00202DE9F8430446002790460E469E
:1000C0008DF800706846FCF7AFFE204600F039F866
:1000D00038B105279DF80000FCF7CAFE3846BDE898
:1000E000F88320680568B8F1000F05D10168204643
:1000F00000F03FF821680860E268012A0CD0022A6B
:100100000ED0042A11D06068082A13D005FB020122
:100110003046FCF7ABF9DDE76068405D3070D9E749
:10012000606830F815003080D4E7606850F825002A
:100130003060CFE700EBC501D1E90001C6E900015D
:10014000C8E7016808684968884201D10120704702
:100150000020704701680A6849688068884201D9B0
:10016000491C00E00021914201D10120704700208C
:1001700070478068884201D9481C7047002070474A
:100180002DE9F84304464FF000080E468DF8008034
:100190006846FCF749FE2046FFF7DCFF07000AD05F
:1001A000207C40B14FF004089DF80000FCF760FE91
:1001B0004046BDE8F8832068456841682046FFF75F
:1001C000D8FF2168486037B1206801682046FFF7F2
:1001D000D0FF21680860E268012A14D0022A16D0F4
:1001E000042A19D0082A1CD06068314605FB020099
:1001F000FCF73CF9204601F06BFA21688A688242DC
:10020000D2D28860D0E7616830784855F2E76168FB
:10021000308821F81500EDE76168306841F8250065
:10022000E8E7D6E90001626802EBC502C2E9000115
:10023000E0E7826800219160826811618268516103
:100240008268D1608268516080680160704708B53B
:10025000002242504058009008BD000020B10349E0
:1002600009680160002070470E2070476C2802006A
:100270002DE9FE4307460E460846FFF7EFFF00282C
:100280007AD100250095019506208DF800704FF079
:100290000108ADF8040002958DF80280694620201F
:1002A00032686ADF3549364A891AC908012202EBE9
:1002B000014430B100F018FA024620463149FFF7F8
:1002C0001DFD00958DF80080019502958DF8018047
:1002D0006946402032686ADF30B100F005FA024614
:1002E00020462949FFF70AFD00958DF80070F72098
:1002F000ADF80200019502956946232032686ADF55
:1003000030B100F0F1F9024620462049FFF7F6FC33
:100310000095019502958DF80080694601203268AC
:100320006ADF30B100F0E0F9024620461849FFF7D5
:10033000E5FC4FF4B0600090019502956946A1205C
:1003400032686ADF30B100F0CFF902462046114929
:10035000FFF7D4FC0095019502958DF80050694691
:10036000A02032686ADF30B100F0BEF902462046B4
:100370000949FFF7C3FC0020BDE8FE8304320200F8
:100380007C310200A02F0200E82F0200343002006E
:10039000002F02004C2F0200AC2E02002DE9F0418C
:1003A0000546076860DF804619491A482A68081A16
:1003B000C608BA4219D9022000EB064416A120460D
:1003C000FFF798FC20463A461FA12B68FFF79DFCDB
:1003D0004FF08050D0F80C012968800200F10050E5
:1003E000421A204625A1FFF789FCB8F100004FF022
:1003F00001040AD000F078F9024604EB06402AA175
:10040000FFF77CFC4046BDE8F0812F480470F9E717
:10041000043202007C310200496E737566666963BE
:1004200069656E742052414D20616C6C6F6361741C
:10043000656420666F722074686520536F6674442B
:1004400065766963652E00004368616E6765207498
:1004500068652052414D207374617274206C6F6323
:100460006174696F6E2066726F6D20307825782018
:10047000746F20307825782E000000004D61786977
:100480006D756D2052414D2073697A6520666F72DB
:10049000206170706C69636174696F6E206973208C
:1004A000307825782E00000073645F626C655F65AC
:1004B0006E61626C6528292072657475726E656460
:1004C0002025732E00000000D32E002030B51548E3
:1004D000ADF5017D0078002821D04FF4FA7500BFFA
:1004E000ADF8005280A9684661DF38B1052816D002
:1004F0000DF5017DBDE83040FCF76EBB6C460A4946
:100500007DA800F083F806E0D0E90021204690475E
:100510007DA800F092F87F980028E1D0F4E70DF56F
:10052000017D30BDD32E0020702802007CB5194C0F
:10053000207808B108207CBD0120A070002001F0C7
:100540002FFB112819D0002001F042FB1248002691
:10055000006801908DF800606846FCF765FC0F4963
:1005600001A810DF05000AD0002020709DF80000CF
:10057000FCF77EFC2DB128467CBD00207CBD01200F
:10058000F3E7A670667001F0BBFB012001F020FBD1
:10059000F3E70000D02E00200428020055CB010014
:1005A0000EB50749684600F031F805E0D0E90010C3
:1005B0008847684600F041F802980028F6D10EBD41
:1005C000202802000148007870470000D02E00204B
:1005D0001FB568464BDF30B1052814D004B0BDE824
:1005E0001040FCF7F9BA084901A800F00FF806E03E
:1005F000D0E900210098904701A800F01EF8039868
:100600000028E6D0F4E71FBD8C28020001600968CD
:100610004160AFF3008010B5D0E9002153689942E2
:1006200001D1002104E0D1E90034A34202D01946EF
:10063000816010BD08314160F0E7816800290BD06E
:10064000026892680A44826041684B689A4203D10A
:1006500008314160FFF7DFBF704770B50D460646B1
:10066000446804E0B2682946904718B124682068BD
:100670000028F7D120682860256070BD40680068B8
:10068000704741680868002801D002680A60704716
:1006900002460020526806E08B4203D108681060D1
:1006A000012070471A461368002BF5D170470000EF
:1006B0000C4A10B502F594730EE0991AC91001EBBB
:1006C000D171491002EBC1010C68844201D90B467B
:1006D00002E005D201F108029A42EED3002010BDDB
:1006E000486810BDA026020000B5FFF7E1FF002812
:1006F00000D1014800BD00008C26020040580028AF
:1007000000D00120704708B50022425040580090A8
:1007100008BDD0F80403084000D0012070474058BD
:10072000002800D00120704708B5002242504058F0
:10073000009008BD02480068002800D001207047E2
:100740000004014008480068012110F0010F06D1A3
:100750004FF0E020C02280F800248430C1670349B4
:10076000012008607047000000E100E0180500402B
:100770000549024600200B790BB1852070470A60BD
:1007800001220A7170470000EC2D0020022010B5F4
:100790004107C1F808034FF48270FEF7DEFD0549FA
:1007A0000120086004480168C1F300410029FAD122
:1007B00010BD00000C00004018040040002802D0CA
:1007C0000149800108477047512602002DE9F04198
:1007D0000D46064600F0F2FD0028304615D0FDF724
:1007E000EFFA083800F06AFE032802D001280AD088
:1007F00003E03046FFF756F828B103213046BDE844
:10080000F041FEF7D1BF0221F8E700F0E3FD002838
:1008100022D03046FDF7D4FA04464FF4807000EB46
:1008200084000E4F81B207EB8400D0F8102542F00F
:100830000102C0F810250846FFF766F8002D0BD01E
:100840003046FDF7BDFA064951F82000002803D0D4
:100850000120A040C7F80403BDE8F081006000401B
:10086000643400202DE9FC41DFF8BC80044608EB2D
:100870000400002790F930001346C0170E46401CB4
:1008800001D008274DE0B0781946C0F34002204659
:10089000FDF772FA0546401C42D0B07841071AD4E1
:1008A000C0070DD068460094FEF7BCFF009900EB2E
:1008B0008101D1F8000720F00200C1F8000707E02D
:1008C00000217378204600910A460191FEF7FBFE55
:1008D000204600F065FDB078800718D513483178C0
:1008E00000EB8500D0F81025114B1A40C0F81025F8
:1008F0004FF47C524FF4403302EA042203EA0141F0
:100900000A43D0F810150A43C0F8102509E008EB97
:100910000500327810F8521F41EA8211017000E0A0
:1009200004273846BDE8FC816434002000600040A4
:10093000FFC0FCFF10B5FEF7B5FF002800D0012076
:1009400010BD000070B5194D95F8640008B108207D
:1009500070BD0024661E2046FEF78EFF10B12819D8
:1009600080F83060641CE4B22A2CF4D300242046C2
:10097000FDF7F4F9641CE4B20C2CF8D3002045F820
:100980005E0F0C49A8800A4CC02081F800040126A3
:100990004020891FC1F800014FF4BE70FEF7B4FF7C
:1009A000A004C4F80403AE71002070BD64340020BC
:1009B0000060004006E000E0034890F86400002872
:1009C00000D0012070470000643400200121B1EB09
:1009D000507F01D1012070470020704738B50D4687
:1009E00000F0DEFD040014D000208DF80000684601
:1009F000FCF71AFA207928B19DF80000FCF738FAC4
:100A0000112038BD0120256020719DF80000FCF701
:100A10002FFA002038BD00000149024801F09EBBBA
:100A2000CC340020002000402DE9F041054600793B
:100A300016460F4600EB40012D4A01EBC00102EBC8
:100A4000810494F82A1011B10820BDE8F0812949E9
:100A500051F820102868FFF7C1FF08B11120F4E712
:100A600039462846FCF71EFA666038692060300077
:100A70004FF001062FD03F7F4FF48E712868FFF7AB
:100A800042FE4FF4A2712868FFF73DFE28681A491C
:100A9000C0F8041328684FEA471140F307300028D4
:100AA00004DB00F1E02080F8001405E000F00F0006
:100AB00000F1E02080F8141D286840F3073000287A
:100AC00009DB00F01F0106FA01F14009800000F186
:100AD000E020C0F8001128680421C0F800150020AB
:100AE000A061E06184F8290044F8140FA675ACE712
:100AF000CC3400200C260200800002002DE9F05FBB
:100B0000054600794FF4017600EB400303EBC0008B
:100B1000344B03EB80040020636813B12B68C3F8E7
:100B20000863A3694FF000096BB1E06938B16068F0
:100B300010B12868C0F804631120BDE8F09FE2619D
:100B40000120216105E0C4F82490A261E160C4F8AD
:100B50001C9094F82910014302D1284600F053FF5D
:100B600060680028286803D0C0F804630020E4E728
:100B70004FF4A2763146FFF7C6FDB2464FF4927BA2
:100B800059462868FFF7BAFD06464FF48471286875
:100B9000FFF7B4FD804651462868FFF7AFFD0746D2
:100BA00048EA07003043EBD056EA070007D1214658
:100BB000286800F0F9FEA169606A8142E0D8C4F8B3
:100BC00018900EB10320B8E70FB10F20B5E794F8E5
:100BD000291001200029296801D00860C6E7486073
:100BE000C4E70000CC3400202DE9F05F0546007911
:100BF0000B4600EB400101EBC000244901EB8004EF
:100C0000284600F045F810B11120BDE8F09F626160
:100C10004FF00009C4F82090A36084F828904FF4A6
:100C20008E784E4641462868FFF76DFD28684FF0E4
:100C3000010AC0F808A02146286801F085F960681B
:100C400008BBD5F800B067690FE000BF94F8280032
:100C500008B10F2615E041465846FFF74FFD002822
:100C6000F4D02146584601F06FF9206AB842F2D319
:100C7000574641462868FFF741FD0028F9D028680B
:100C8000C760C4F814903046BFE70000CC340020A1
:100C9000007900EB400101EBC000044901EB80004A
:100CA0004069002800D0012070470000CC340020AB
:100CB0000149024801F000BBF83400200020004048
:100CC0002DE9F0410546164600790F46154A00EB1E
:100CD000C00102EB810494F8201011B10820BDE896
:100CE000F081114951F820102868FFF777FE08B10C
:100CF0001120F4E739462846FCF70FF96660386999
:100D000020601EB1397F2846FDF73CFD2868082188
:100D1000C0F800150020A061E0616061012184F845
:100D20002010DCE7F8340020102602002DE9F05FE7
:100D3000044600790E4600EBC001DFF8F0A017462C
:100D40000AEB81053046FFF741FEB0B168684FF00D
:100D500000084FF4047910B12168C1F80893A8691C
:100D60004FF0000B80B1E86948B1686810B12068A5
:100D7000C0F804931120BDE8F09F1020FBE7EF615D
:100D80004FF001082E6102E0EE60C5E9067B002508
:100D90004FF488712068FFF7C7FC4FF4A2712068F8
:100DA000FFF7C2FC2068C0F83465C0F838752068C9
:100DB000B8F1000F12D0D0F8001241F02001C0F8B5
:100DC00000122079D04600EBC0010AEB8100406898
:100DD00038B12068C0F804932846CCE701210160AF
:100DE000EFE74FF4887A4FF4A27951462068FFF775
:100DF00096FC074649462068FFF791FC06464FF4EB
:100E000092712068FFF78BFC014647EA0600084311
:100E1000EBD0227902EBC20308EB8302C2F818B0D0
:100E200001B10325002ED7D00F25D5E7F8340020D7
:100E30002DE9F04704460E460079274900EBC00033
:100E400001EB800517463046FFF7C0FD30B1204664
:100E500000F044F820B11120BDE8F0871020FBE736
:100E60006F61AE604FF490774FF00008394620680C
:100E7000FFF75AFC4FF4AC7631462068FFF754FC7C
:100E80002068AA686969C0F84425C0F84815206838
:100E90004FF00109C0F808906868D0B9BA465146C9
:100EA0002068FFF73CFC074631462068FFF737FC17
:100EB0000743F4D010B14FF00F0808E02068C0F8E5
:100EC0000C9031462068FFF72AFC0028F9D000205A
:100ED00068614046C0E70000F83400200079054909
:100EE00000EBC00001EB80004069002800D0012029
:100EF00070470000F8340020FBF76EBE2DE9F84F74
:100F000005460C460888B5F8CA12884279D195F88A
:100F1000C6024FF0000A00EB8001C1EB801005EB28
:100F200040066088002860D13079E288A71D81469C
:100F3000D1B250FA82F2062A02D80844307111E088
:100F400006203071374838493288401AC1080220DB
:100F500000EB014080463549FEF7D0FE404634495B
:100F6000FEF7C8FE48460022D0461BE000EBC00159
:100F700002EB820307EB430306EB4101D3F802C007
:100F8000C1F80AC0D3F806C0C1F80EC05B894B8215
:100F9000A1F81480A1F81680A1F81880401CA1F8CF
:100FA0001A80521C31798142E0D895F8C61200EBC4
:100FB000C00001EB8102C2EB811105EB410136F863
:100FC00010000989884210D2307906280DD085F8A2
:100FD000C50221882846FCF7FBFE002811D0228894
:100FE0002946BDE8F84FFDF75FB885F8C5A222880D
:100FF00069462846FCF766FF28B122882946FDF796
:1010000053F8BDE8F88F9DF800000028F9D0228839
:1010100001212846FCF7EEFF2188284600F072F9EE
:10102000EFE700007C3102007C3102002029020041
:101030006829020070B502468888C97B02EBC004AB
:10104000A41D022901D15188218021886288914202
:1010500013D9A5DF012578B111280FD0FFF744FB84
:10106000024607480749401AC00805EB0040BDE8A2
:10107000704005A1FEF742BE657170BD257170BD5F
:10108000843102007C31020073645F626C655F67CB
:10109000617474635F65786368616E67655F6D74C2
:1010A000755F726571756573742829207265747532
:1010B000726E65642025732E00000000F8B50546A9
:1010C0000C460888B5F8CA12884255D195F8C60270
:1010D000A21D00EB8001C1EB801005EB400695F8E6
:1010E000C50200EBC00006EB400160880A3138B34E
:1010F00029E000BF00EB400302EB43039F88B7F5F4
:10110000245F0CD06FF4245C17EB0C070AD0012F7E
:1011100002D0072F0BD108E05B884B8107E05B888A
:101120008B8104E05B88CB8101E05B880B824B897B
:101130002BB18B891BB1CB890BB10B8A1BB9401C1E
:1011400013888342D6D800208DF8000095F8C50298
:101150003179401C884203D101208DF8000010E055
:1011600085F8C502228869462846FCF7ABFE20B107
:1011700022882946FCF798FFF8BD9DF8000000285A
:10118000FAD0228801212846FCF734FF218828461E
:1011900000F0B8F8F8BD00007CB506468D88C88818
:1011A00006EBC504A41D172800D217202188814210
:1011B00000D8084660800020207121882846B5DFCD
:1011C00060B1FFF791FA02460F481049401AC00873
:1011D000012101EB00400EA1FEF790FD607900288F
:1011E00010D1306900280DD01549D1E90201CDE9AF
:1011F0000001ADF802506088ADF80400326969461C
:10120000304690477CBD0000843102007C310200F2
:1012100073645F626C655F67617474735F65786344
:1012200068616E67655F6D74755F7265706C792853
:10123000292072657475726E65642025732E000016
:10124000CC25020070B505460C4690F8C6022288EF
:1012500000EB8001C1EB801005EB4001B5F8CA023C
:10126000824238D1608848B100212846FCF7C2FE8E
:1012700021882846BDE8704000F044B8E268C1F813
:101280000620E28895F8C412D0B251FA82F2062AFA
:1012900003D8084485F8C40211E0062085F8C4028A
:1012A0000D480E49401AC108022000EB01460CA16E
:1012B0003046FEF71FFD30461149FEF71BFD218821
:1012C0002846FCF785FD002805D022882946BDE880
:1012D0007040FCF7E9BE70BD7C3102007C31020039
:1012E0004E6F7420656E6F756768207370616365FB
:1012F00020666F722073657276696365732E0000D5
:10130000C429020070B588B00D4604462021684605
:10131000FBF7C5F894F8C7021E4B401CC0B284F816
:10132000C702DA68002190422CD284F8C51294F8E2
:10133000C602194E401CC2B202EB820084F8C622DB
:10134000C0EB821006EB820204EB400012680260E0
:10135000017102218DF800100121ADF81010006814
:10136000CDF812000D48CDE902042A466946986876
:10137000FDF7B0FD002803D02A462146FCF794FE75
:1013800008B070BD84F8C81229462046FCF71AFE42
:10139000F6E70000C82D002038340020A9E0010045
:1013A00010B50549C20800F00703885C01249C4081
:1013B0002043885410BD0000C23400200449084472
:1013C00090F93000082801DB0120704700207047A9
:1013D000643400200449084490F93000082801D200
:1013E0000120704700207047643400202DE9F84F39
:1013F000314F05464FF001090024381990F95A1071
:10140000491C46D090F85A00294620F0C0063046C4
:10141000FDF789FC70B3204600F050F8824668461C
:101420000096FEF7FFF9009900EB8100D0F8000765
:10143000C0F30148B8F1020F1DD002213046FEF77B
:10144000B3F968460096FEF7EDF9009A09FA02F141
:10145000C0F820153046FCF7B3FC57F820204AB1FD
:101460005046BAF1030F11D0B8F1020F05D0B8F110
:10147000030F07D00DE00321E0E75046BAF1010F5A
:1014800004D006E05046BAF1020F02D101463046C0
:101490009047641C042CB0D32A4602210020FEF79A
:1014A0009BF9002055F820100029A5D1401C0228E6
:1014B000F8D3BDE8F88F00006434002002490844E6
:1014C00090F85A00800970476434002010B50C462B
:1014D000017A052908D0407A38B1084808A1026885
:1014E0002046FDF7D1FF00E01AB106A12046FDF726
:1014F000CBFF2046BDE81040FDF7D3BFAC2E002047
:10150000257300000D0A000038B5C3880D46044657
:1015100033B114A0009015A216A12846FDF7B4FF20
:10152000217A05291CD0607A48B1A088FEF7A0FA7C
:10153000164951F8202016A12846FDF7A5FFA088DE
:101540000021FEF777FC03461049207A143951F840
:10155000202001B02846BDE830400EA1FDF794BF21
:1015600038BD00001B5B306D000000001B5B313B91
:1015700033316D0025734C6F67732064726F707028
:101580006564202825642925730D0A00AC2E0020EF
:10159000257300003C25733E2025733A200000008F
:1015A0000349884201D1034870470020704700007A
:1015B00000200040F42D0020F0B591B00E46074603
:1015C00001226946FEF776FD04005AD19DF800001D
:1015D00004AD06285DD2DFE800F0030A181F2327B8
:1015E000BDF81220BDF810103046A1DF0BE00CA8AA
:1015F00006900146BDF8162000230198FEF7F5FC81
:1016000029463046A3DF044626E0BDF810103046D8
:101610000DF112029BDFF6E7294630469DDFF2E727
:10162000294630469EDFEEE70CA8079000230222F1
:1016300008A90198FEF7D9FC08A80690BDF820205B
:10164000022307990198FEF7D0FCBDF820E0294657
:101650003046AEDF040016D0112C12D09DF80000E9
:10166000114951F8200010B10198FEF790FC0022BA
:1016700069463846FEF71EFD22463146684600F0B0
:101680007BF811B0F0BDBDF820008645E6D00C24F3
:10169000E4E706480649401AC008022101EB004071
:1016A00004A1FEF727FBD9E7DC2502008C310200FC
:1016B0007C310200556E696D706C656D656E746588
:1016C000642047415454205265717565737400005D
:1016D00001680A684968914201D3881A7047806896
:1016E000801A0844401C704770B58CB00446C0682E
:1016F000002209A9FEF7DEFC104D1BE0BDF8241006
:10170000A06801EB810100EB810607E09DF8000075
:1017100055F8200010B10198FEF739FC0022694607
:101720003046FEF7C7FC0028F0D0002209A9E06887
:10173000FEF7C0FC0028E1D00CB070BDDC25020033
:1017400070B50C4B00210A4ADC680DE002EB810504
:101750008678AD78B54206D132F821500688B54278
:1017600001D1586870BD491CA142EFD3002070BD63
:1017700038340020C82D0020F8B515000E46044668
:1017800016D00C480C490095401AC008012101EB05
:101790000040227833460949FEF7BFFAA368002BC0
:1017A00006D0E16801B032462846BDE8F04018474F
:1017B000F8BD00008C3102007C3102000C2A0200CE
:1017C0002DE9F041044600780E46002504F1100191
:1017D000062828D2DFE800F003080B111418628AEB
:1017E000218A3046A1DF0DE03046A3DF0AE0218ADE
:1017F00004F1120230469BDF04E030469DDF01E039
:1018000030469EDF054605E0A06907883046AEDF1A
:10181000050002D0112D18D00FE0A0690088B84251
:101820000BD00C2509E00A480A49401AC0080221D9
:1018300001EB004008A1FEF75DFA2A46314620463A
:10184000FFF79AFF0120BDE8F0810020FBE70000D0
:101850008C3102007C310200556E696D706C656DD3
:10186000656E7465642047415454205265717565F6
:101870007374000070B50546FCF743FD134C40B18E
:10188000D4E904024FF08071411842F10000C4E92C
:10189000041000212846FCF781FC30B1606820B1BB
:1018A000606800F0C1FA0020606001212846FCF762
:1018B00075FC18B1FCF7DAFEC4E90601284600F011
:1018C000DFFA2846BDE8704000F034B8182E00203A
:1018D00070B5054600200C460870FCF7C7FED5E938
:1018E0000223101A63EB010300263146361A994190
:1018F00012DAB0F5350F03D3FBF7A2F90B49421802
:101900004FF4960300210A48FCF707FD10B10D289B
:1019100006D009E0012070BD00210548FCF734FC29
:10192000284600F081FA2070002070BDFFFFB4004F
:10193000202E0020F8B51A4C074600261948FEF75D
:101940009DFED0B1616871B1D0E902106268D2E940
:101950000232C91A904120D26068007F18B16168D4
:101960001048FEF77AFE00F0F7F905466946FFF7E2
:10197000AFFF98B1606840B10AE0606800280CD100
:101980003846BDE8F840FCF7C4BC3846FCF7BDFC5F
:1019900065609DF800000028D0D1F8BD6660CDE7F5
:1019A000182E00202426020070B5054688690C46D2
:1019B00000284FF4847128460AD0FEF7A4FED5F81B
:1019C0001805626AE1688854606A401C606270BDF4
:1019D000FEF799FED5F8180570BD1FB501238DF8E7
:1019E0000030CDE90121D0E90012684690471FBDC3
:1019F0001FB501238DF80030CDE90121D0E9001297
:101A0000684690471FBD10B5044600684FF49271B8
:101A1000FEF779FE4FF484712068FEF774FE2068AB
:101A20000121016010BD00007FB501460378144814
:101A3000144A801AC008032202EB0040042B18D07D
:101A4000052B0ED0062B0BD14968CA788D794C79BD
:101A50000B798DE83C008B784A780BA1FEF766F98C
:101A60007FBD48680028FBD004B0BDE87040FBF79C
:101A7000B3B811A1FEF73EF9BDE87F4000F050B8C1
:101A8000F43102007C310200436F6E6E656374694D
:101A90006E6720746F207461726765742025303220
:101AA000782530327825303278253032782530323A
:101AB00078253032780000005363616E2074696DC0
:101AC0006564206F75742E001FB500200090019092
:101AD0000290039001208DF804008DF80C000D4A4F
:101AE00069460D48FDF7FBFA08B1FBF775F80B4A9C
:101AF00003210948FDF7B0FA08B1FBF76DF80022A1
:101B000004210548FDF7D0FA002801D0FBF764F85E
:101B10001FBD0000291A0200F83100200025020034
:101B200010B50848FDF7CEFB08B1FBF755F80120CA
:101B3000FBF750FF002803D0BDE81040FBF74CB87E
:101B400010BD0000F831002038B50021012548B152
:101B5000012810D003280DD1FEF7F4FDBDE8384070
:101B6000FDF724BC4FF0E020C0F88051BFF34F8F49
:101B7000BFF36F8F38BD8DF800106846FBF754F93E
:101B8000064C207808B9FDF7F1FBE068401CE060E6
:101B9000A5709DF80000FBF76BF938BD50340020AC
:101BA0003EB5044609496846FEF730FD08E000BF2F
:101BB000D0E900212046904730B16846FEF73DFD50
:101BC00002980028F4D13EBD11203EBD0828020035
:101BD0003EB5044608496846FEF718FD07E000BF19
:101BE000D0E90021204690476846FEF726FD02987E
:101BF0000028F5D13EBD0000142802002DE9F04177
:101C00001400884618D000250E4F032608EB050166
:101C100022460020FAF73EFD0544241A40B93878E0
:101C2000002809D008494FF47A408847761E05D02D
:101C300001203870002CE9D1BDE8F0810020387017
:101C4000FAE70000702E0020E127020010B50446DC
:101C50000020FBF7BFFE08B1FAF7BEFF24B9FBF77F
:101C600025FE08B1FAF7B8FF012010BD70B5194D77
:101C7000194C07E0016820788847002829D01548CA
:101C8000FEF7DBFCA8680028F4D1FEF7E1F800BFFE
:101C9000FDF714FF0028FBD1207803280CD0022880
:101CA0000AD0FEF78FFC00B133DF0C490120086039
:101CB000BFF34F8F20BFFDE7BFF34F8F0848016888
:101CC000084A01F4E06111430160BFF34F8F00BF88
:101CD000FDE770BDF4350020642E002000050040B3
:101CE0000CED00E00400FA05002805D103490120AD
:101CF00048700020FCF7A2B8704700005034002064
:101D000010B51620FAF792FEA0B1114890F8000421
:101D10004009082811D20121814011F0EC0F0CD0AC
:101D20000C4882684FF480016AB1016841F4800177
:101D3000016010BD42F2010001E042F20200BDE884
:101D40001040FAF749BF4FF0E020C0F8001110BD75
:101D500016E000E0E83500200148FEF792BC0000E4
:101D600024260200C207002A03D000BF4FF00F0252
:101D700001E04FF0F00201D04FEA0111044B03EBF8
:101D80005003187800EA020040EA0100187070471A
:101D9000403500202DE9F84F0746214891468846F6
:101DA00005681E46012269461846FBF751FFDFF819
:101DB00074A060B3009800210446801C0AE000BFB4
:101DC00000EA050259F821C00AEB8202401C491CB6
:101DD000C2F80CC0B142F3D34FEA1749FCF7CAF975
:101DE000611C29400AEB810149EA00422C40CA608B
:101DF0000AEB8401C86867F3C50066F3891068F3CD
:101E00009F2020F00300401C20F00400C8609AF8D6
:101E1000000001E0FDF752FE0028FBD1BDE8F88F7D
:101E20007C2E00209837002070B50446124800250B
:101E30000078F8B1F4B1207FE0B1FCF717FCD4E9E9
:101E40000223801A994110D32069002600B9267711
:101E5000D4E905108847206960B1217F51B1D4E9E8
:101E6000022110187141C4E9020121460348FEF71E
:101E7000F4FB0125284670BD182E00202426020000
:101E8000F8B51B4C69462068FCF7C3FE0026012705
:101E9000184D29E0017821B101290CD002291BD16C
:101EA00014E041680A7FBAB90F77416810480830DA
:101EB000FEF7D3FB10E041686868814201D16E6093
:101EC0000AE00B480830FEF7E3FB05E0FFF744FFAC
:101ED00008B10677FAE72F7069462068FCF78EFE96
:101EE00069462068FCF795FE0028D3D1F8BD0000B4
:101EF0001C260200182E0020F8B50B4C0D46064695
:101F000069462068FCF76FFE58B106704560694667
:101F10002068FCF789FE10B10448FCF7DFF90020C7
:101F2000F8BD0420F8BD00001C260200202E002071
:101F3000034880684108034800224068FAF7C0BEA1
:101F4000002E00201426020070B50C4605464FF402
:101F50008E71FEF7D8FB216AA068415C206A401CA4
:101F60002062C5F81C1570BD1FB500228DF8002039
:101F70000291816801914261D0E900126846904760
:101F80001FBD1FB500228DF80020029181680191CC
:101F90004261D0E90012684690471FBD70B50278D3
:101FA000044662B11C481D4B0121C01AC00801EB58
:101FB0000040012A27D0022A24D119A124E0264C6E
:101FC000244D60882844FAF799FE6088401C80B24E
:101FD0002918608011F8011C0A2904D00D2902D0AB
:101FE000218888420ED31B49628801F53D70FBF7BA
:101FF0009FFA082804D01328F5D008B1FAF7ECFDB1
:102000000020608070BD15A1FDF774FE6068BDE81A
:102010007040FAF7E1BD0000F43102007C310200AB
:10202000436F6D6D756E69636174696F6E20657263
:10203000726F72206F63637572726564207768696E
:102040006C652068616E646C696E672055415254FE
:102050002E000000D82E0020B02700204572726F9D
:1020600072206F6363757272656420696E204649E1
:10207000464F206D6F64756C6520757365642062D2
:102080007920554152542E007CB50178254DA1B3DD
:1020900001290BD002291DD18DF80010C068691CE0
:1020A00001900122C81DFDF7CFF930E0017A59B146
:1020B000406801781C48FAF7B5FD1B4C012650B169
:1020C0008DF8006001900DE016490122491CC81DE1
:1020D000FDF7BAF97CBDA068E168814205D0002017
:1020E0008DF80000696868468847A068E168081AAA
:1020F000A1888842E8D9AE707CBDFFE70A4809494B
:102100001030FAF774FD30B103208DF800006968D3
:1021100068468847F0E70349012201F10800FDF70E
:10212000A3F9E9E73C2E0020C83500201FB50A4678
:1021300001788DF8001041680191017A8DF808103E
:10214000C0680390044850F82210083850F8222044
:10215000684690471FBD0000E42D00202DE9FF4791
:102160000C4605464FF40071FEF7D3FA01274FF4F1
:102170000178002618B34FF4927949462846FEF7B5
:10218000BDFAE0B149462846FEF7BDFAC5F8088316
:1021900094F8290000B96F6002208DF80000D5F88E
:1021A0008004C5F880040390A0690290E068019063
:1021B000A661E661D4E900126846904728E0042150
:1021C0002846FEF7A6FA18B34FF484712846FEF7A6
:1021D00095FAE8B121462846FFF7E6FB616AA06957
:1021E000884215D1E06938B1E268616AA06120696E
:1021F000E6616662E06008E094F8290000B96F606B
:10220000C5F80883A661E268616A2046FFF7E5FB2E
:102210004FF48E7841462846FEF770FA80B1606927
:10222000216A814202D294F8280028B34146284608
:10223000FEF769FA606918B161692046FFF794FEFC
:102240004FF4A27841462846FEF758FA002818D0E5
:1022500041462846FEF757FA94F8290000B12F604E
:10226000A06900280DD0A661E268616A04B020462A
:10227000BDE8F047FFF7B1BB21462846FFF764FEF3
:10228000DEE7BDE8FF8700001FB50A4601788DF83C
:10229000001041680191017A8DF80810C068039020
:1022A000044850F82210083850F822206846904719
:1022B0001FBD0000E42D00202DE9FF410C464FF426
:1022C000927705463946FEF72AFA0026B8B1394614
:1022D0002846FEF729FA02208DF80000D5F8800480
:1022E000C5F880040390D5F83C050290E0680190A1
:1022F000A661E661D4E900126846904723E04FF4F6
:10230000887739462846FEF70AFAE0B1394628466A
:10231000FEF70AFAD5F83C15A069884213D1E069A6
:1023200060B1E268D5F8000220F02000C5F8000294
:10233000E069A0612069E661E06001E0A661E26811
:102340002046FFF755FB4FF4A27739462846FEF7A3
:10235000E6F968B139462846FEF7E6F9A06938B1D2
:10236000A661E661D5F83C152046E268FFF740FB20
:102370004FF4907631462846FEF7D1F960B13146E8
:102380002846FEF7D1F90120E860606920B1D5F850
:102390004C152046FFF7F5FD4FF4AC763146284644
:1023A000FEF7BDF900280ED031462846FEF7BCF9ED
:1023B0006069002807D0D5F84C1504B02046BDE868
:1023C000F041FFF7DEBDBDE8FF8100002DE9F05FC1
:1023D0008346DDE90A4A994690460D46084601279C
:1023E00003E000BFB0FBF8F07F1C4045FAD2B945CE
:1023F00000D94F465FEACA7012D18CB15FEA8A7089
:1024000002D5B9F1000F01D0202607E0302605E003
:1024100031465846641EFBF765FC0CB1A742F7D362
:102420005FF00106B9F1010F02D9A9F1010903E03A
:10243000B5FBF6F0404502D306FB08F6F2E7DFF8FD
:102440003C9000BFB5FBF6F000FB165519F80010E4
:102450005846FBF747FCB6FBF8F6002EF2D15FEAD0
:10246000CA7009D0002C07D0A74205D220215846B7
:10247000641EFBF737FCF5E7BDE8F09F5626020027
:1024800070B50C460546FBF751FC002807D04268A2
:10249000002A04D021462846BDE87040104770BD90
:1024A00010B504281DD209B1032400E00024FBF775
:1024B0003FF9202802D24FF0A04102E00A4900F083
:1024C0001F0001EB8000D0F8001721F44031C0F864
:1024D0000017D0F8001741EA0441C0F800170020A7
:1024E00010BD062010BD000000030050EC3200209B
:1024F0004C32002004000000200000000100000019
:1025000001000200080000000600000005000000B5
:10251000070000000000000000E0D7010D0E0F10C2
:102520000B0C1819C8330020E833002018340020A1
:102530000B000300CDD801000C000300CDD8010032
:1025400018000300CDD8010019000300CDD8010008
:10255000010000000000000000000000000000007A
:10256000000000000000000000000000000000006B
:10257000000000000000000000000000000000005B
:10258000000000000000000000000000000000004B
:10259000000000000000000000000000000000003B
:1025A000000000000000000000000000000000002B
:1025B000000000000000000000000000000000001B
:1025C000000000000000000000000000770A00008A
:1025D00000000000770A000000000000000000007A
:1025E00001E6010000000000000000000000000003
:1025F0002DE601009ECADC240EE5A9E093F3A3B505
:102600000000406E0000005000030050190A020054
:10261000B10C0200030000002035002060350020CE
:102620000100060000000000382E002081DE0100BD
:10263000FFFFFFFFFFFFFFFFFFFFFFFFFFFFFFFFAA
:1026400000000000000000000000D60106010000AC
:102650000338FDD8704730313233343536373839A6
:1026600041424344454600000000000000000000D5
:10267000503202005432020000000000000000004E
:10268000682602008026020004000000556E6B6E72
:102690006F776E206572726F7220636F64650000E1
:1026A00000000000D02D0200010000007C2C020080
:1026B00002000000702A020003000000F02C02005B
:1026C00004000000442D020005000000242C02003C
:1026D00006000000C02B0200070000002C2D0200A5
:1026E00008000000382C0200090000009C2C0200A9
:1026F0000A000000B82D02000B000000582A02005A
:102700000C000000502C02000D000000202E0200E2
:102710000E0000001C2D02000F000000582D0200CA
:10272000100000008C2D020011000000342E020069
:1027300012000000082E020013000000A42D020069
:1027400080000000D82B020081000000142B020042
:1027500082000000D42A020083000000B42A020094
:1027600084000000F02A020085000000FC2B02001B
:1027700086000000042D020090000000A02B020043
:1027800091000000942A020092000000642C0200D4
:10279000008200006C2D020001820000B82C0200B3
:1027A00002820000D42C020000840000302B0200C2
:1027B00001840000DC2D020002840000782B02005E
:1027C00003840000542B020091F901008FF90100ED
:1027D00089F9010000000000000000000000000076
:1027E0000338FDD870470000003700207F0000004C
:1027F0008037002000000000000000000000000002
:102800000000000001000007F42702000428020075
:10281000080000002C2802003C28020008000000EC
:102820003C2802004C28020008000000A4320200EC
:10283000AC320200000000000000000094320200F0
:10284000A4320200000000000000000000000000B0
:1028500000000000543202007C3202007C32020090
:1028600084320200843202008C320200B027002041
:102870004C2802006C280200080000008C32020084
:102880009432020000000000000000007C280200DA
:102890008C280200080000000040404040404040BA
:1028A0004040414141414140404040404040404023
:1028B00040404040404040404005020202020202C7
:1028C0000202020202020202022020202020202016
:1028D000202020020202020202029090909090902A
:1028E00010101010101010101010101010101010E8
:1028F000101010100202020202028888888888885C
:102900000808080808080808080808080808080847
:10291000080808080202020240000000992802008C
:102920004E6F7420656E6F756768207370616365A4
:1029300020666F7220636861726163746572697387
:1029400074696373206173736F6369617465642074
:1029500077697468207365727669636520307825BD
:102960003034582021000000496E63726561736540
:1029700020424C455F474154545F44425F4D4158AB
:102980005F434841525320746F2062652061626C3E
:102990006520746F2073746F7265206D6F7265208F
:1029A00063686172616374657269737469637320CB
:1029B000666F72206561636820736572766963650E
:1029C00021000000496E63726561736520424C45C9
:1029D0005F44425F444953434F564552595F4D410E
:1029E000585F53525620746F2062652061626C6597
:1029F00020746F2073746F7265206D6F7265207321
:102A000065727669636573210000000053442047B6
:102A10004154542070726F63656475726520282577
:102A20006429206661696C6564206F6E20636F6E37
:102A30006E656374696F6E2068616E646C652025D5
:102A4000642077697468206572726F723A203078FA
:102A5000253038582E0000004E52465F4552524FE6
:102A6000525F494E56414C49445F44415441000035
:102A70004E52465F4552524F525F534F4654444563
:102A8000564943455F4E4F545F454E41424C454485
:102A9000000000004E52465F4552524F525F46457D
:102AA00041545552455F4E4F545F454E41424C454F
:102AB000440000004E52465F4552524F525F4D5502
:102AC0005445585F554E4C4F434B5F4641494C452A
:102AD000440000004E52465F4552524F525F4D55E2
:102AE0005445585F4C4F434B5F4641494C45440069
:102AF0004E52465F4552524F525F4D555445585FB6
:102B0000434F4E445F494E49545F4641494C45440A
:102B1000000000004E52465F4552524F525F4D55E5
:102B20005445585F494E49545F4641494C4544001D
:102B30004E52465F4552524F525F424C455F49509C
:102B400053505F52585F504B545F5452554E43415F
:102B5000544544004E52465F4552524F525F424CDC
:102B6000455F495053505F504545525F52454A4575
:102B700043544544000000004E52465F4552524FB8
:102B8000525F424C455F495053505F4C494E4B5F3A
:102B9000444953434F4E4E454354454400000000C2
:102BA0004E52465F4552524F525F4150495F4E4F21
:102BB000545F494D504C454D454E5445440000002E
:102BC0004E52465F4552524F525F4E4F545F5355DF
:102BD00050504F52544544004E52465F4552524F5A
:102BE000525F4D4F44554C455F4E4F545F494E49DF
:102BF0005449414C495A4544000000004E52465F3A
:102C00004552524F525F4D4F44554C455F414C52D7
:102C1000454144595F494E495449414C495A4544FC
:102C2000000000004E52465F4552524F525F4E4FD9
:102C3000545F464F554E44004E52465F4552524FE8
:102C4000525F494E56414C49445F535441544500EC
:102C50004E52465F4552524F525F444154415F537A
:102C6000495A45004E52465F4552524F525F494FB6
:102C70005F50454E44494E47000000004E52465FAB
:102C80004552524F525F5356435F48414E444C4564
:102C9000525F4D495353494E470000004E52465F24
:102CA0004552524F525F494E56414C49445F4C4544
:102CB0004E475448000000004E52465F4552524F66
:102CC000525F4452565F5457495F4552525F414EDE
:102CD00041434B004E52465F4552524F525F445261
:102CE000565F5457495F4552525F444E41434B0033
:102CF0004E52465F4552524F525F494E5445524ED6
:102D0000414C00004E52465F4552524F525F535461
:102D10004F524147455F46554C4C00004E52465F6E
:102D20004552524F525F4E554C4C00004E52465F3A
:102D30004552524F525F494E56414C49445F5041B3
:102D400052414D004E52465F4552524F525F4E4FD8
:102D50005F4D454D000000004E52465F4552524FB8
:102D6000525F464F5242494444454E004E52465FE0
:102D70004552524F525F4452565F5457495F455235
:102D8000525F4F56455252554E0000004E52465F1C
:102D90004552524F525F494E56414C49445F41445F
:102DA000445200004E52465F4552524F525F5245C8
:102DB000534F5552434553004E52465F4552524F72
:102DC000525F494E56414C49445F464C414753007F
:102DD0004E52465F53554343455353004E52465F50
:102DE0004552524F525F424C455F495053505F43EA
:102DF00048414E4E454C5F414C52454144595F4518
:102E000058495354530000004E52465F4552524FAA
:102E1000525F434F4E4E5F434F554E5400000000EB
:102E20004E52465F4552524F525F54494D454F55A1
:102E3000540000004E52465F4552524F525F425579
:102E4000535900007761726E696E67006465627540
:102E5000670000001B5B313B33306D001B5B306D46
:102E6000000000001B5B313B33316D001B5B313BCD
:102E700033326D001B5B313B33336D001B5B313BE9
:102E800033346D001B5B313B33356D001B5B313BD5
:102E900033366D001B5B313B33376D00696E666FF7
:102EA000000000006572726F7200000073645F6260
:102EB0006C655F6366675F7365742829207265744B
:102EC00075726E6564202573207768656E20617465
:102ED00074656D7074696E6720746F2073657420FB
:102EE000424C455F47415454535F4346475F534507
:102EF00052564943455F4348414E4745442E0000E2
:102F000073645F626C655F6366675F7365742829CD
:102F10002072657475726E6564202573207768650C
:102F20006E20617474656D7074696E6720746F20B3
:102F300073657420424C455F434F4D4D4F4E5F4388
:102F400046475F56535F555549442E0073645F6290
:102F50006C655F6366675F736574282920726574AA
:102F600075726E6564202573207768656E206174C4
:102F700074656D7074696E6720746F20736574205A
:102F8000424C455F47415454535F4346475F415469
:102F900054525F5441425F53495A452E000000008D
:102FA00073645F626C655F6366675F73657428292D
:102FB0002072657475726E6564202573207768656C
:102FC0006E20617474656D7074696E6720746F2013
:102FD00073657420424C455F434F4E4E5F434647F6
:102FE0005F4741502E00000073645F626C655F6351
:102FF00066675F73657428292072657475726E65E3
:1030000064202573207768656E20617474656D7027
:1030100074696E6720746F2073657420424C455F3D
:103020004741505F4346475F524F4C455F434F55C2
:103030004E542E0073645F626C655F6366675F73F6
:10304000657428292072657475726E656420257315
:10305000207768656E20617474656D7074696E6741
:1030600020746F2073657420424C455F434F4E4E71
:103070005F4346475F474154542E0000626C655FD2
:1030800064625F64697363006E72665F626C655F41
:1030900067617474000000006E72665F626C655F49
:1030A00067710000626C655F7363616E0000000011
:1030B000626C655F6E75735F63000000636C6F63C5
:1030C0006B000000434C4F434B0000004750494FFA
:1030D0005445000050525300554152540000000026
:1030E00055415254450000006170705F6275747400
:1030F0006F6E00006170705F74696D657200000032
:103100007077725F6D676D7400000000736F72748A
:103110006C697374000000007274745F6C6F675F99
:103120006261636B656E6400617070006E72665FF1
:10313000736468006E72665F7364685F626C6500DA
:103140006E72665F7364685F736F6300AC32020017
:10315000B02700202807000034C501001433020006
:10316000D82E0020681700001CCA0100C8270200E2
:103170000000000018310200742E00207C30020094
:1031800000000303883002000000030398300200AF
:1031900000000303A430020000000303B03002006B
:1031A00000000303BC30020000000000C430020035
:1031B00000000000CC30020000000000D43002000B
:1031C00000000000D830020000000000E0300200E3
:1031D00000000000E830020000000000F4300200AF
:1031E0000000000000310200000000000C3102006D
:1031F0000000000028310200000003032C3102000F
:1032000000000303343102000000030340310200D8
:1032100000000303A82D00209E2D0020A62D0020D5
:103220000433002018000000882E0020802E00208B
:10323000882E00204036002018000000F8320020C0
:103240009A2D002001000000020000000100000093
:103250004D1C020071ED0100E4310020F1D00100AD
:10326000B427002045F20100F831002075EF01007D
:10327000842D002095D201000000000045D40100FB
:10328000CC31002075D1010000000000E91C0200D3
:1032900000000000CD04020000000000D105020083
:1032A00000000000491B02000000000002FF1401A2
:1032B000FF01CF03FFFFFF01FF01FF7132011398F0
:1032C0002D1520EC2402143C32021A14040387FF4B
:1032D000FF15100140110222041220BA4008011FFC
:1032E00029DF091EE314A42E021A44041A9C041AAE
:1032F0004C041A5C041A54041A64041A6C041A74F8
:10330000041A7C041A84041A8C041A9404510400CC
:0433100090D0030056
:040000050001C20133
:00000001FF
